:020000040000FA
:0408000064EF0BF0A6
:1008100003B273EF05F0F2B491EF05F09EB099EFDB
:1008200005F09EB2A1EF05F0F2A81AEF04F0F2B2C3
:1008300021EF04F0F2B01FEF04F013EF0BF0F2968B
:10084000F290CD90F2929EA02BEF04F00101533F65
:100850002BEF04F0542BB2C1B6F1B3C1B7F1B4C160
:10086000B8F1B5C1B9F1AEC1B2F1AFC1B3F1B0C128
:10087000B4F1B1C1B5F1AAC1AEF1ABC1AFF1ACC138
:10088000B0F1ADC1B1F1A6C1AAF1A7C1ABF1A8C148
:10089000ACF1A9C1ADF1A2C1A6F1A3C1A7F1A4C158
:1008A000A8F1A5C1A9F19EC1A2F19FC1A3F1A0C168
:1008B000A4F1A1C1A5F19AC19EF19BC19FF19CC178
:1008C000A0F19DC1A1F1CECF9AF1CFCF9BF153C141
:1008D0009CF154C19DF1CF6ACE6A0101536B546BF8
:1008E0009E90CD800FBC0F8E0FBA7AEF04F00F8A66
:1008F00013EF0BF013880F8C0FBEB7EF04F09AC103
:100900009EF19BC19FF19CC1A0F19DC1A1F19EC12F
:10091000A2F19FC1A3F1A0C1A4F1A1C1A5F1A2C1FF
:10092000A6F1A3C1A7F1A4C1A8F1A5C1A9F1A6C1CF
:10093000AAF1A7C1ABF1A8C1ACF1A9C1ADF1AAC19F
:10094000AEF1ABC1AFF1ACC1B0F1ADC1B1F1AEC16F
:10095000B2F1AFC1B3F1B0C1B4F1B1C1B5F1B2C13F
:10096000B6F1B3C1B7F1B4C1B8F1B5C1B9F1010184
:100970005E6B5F6B606B616B9A515E279B515F236F
:100980009C5160239D5161239E515E279F515F239F
:10099000A0516023A1516123A2515E27A3515F237F
:1009A000A4516023A5516123A6515E27A7515F235F
:1009B000A8516023A9516123AA515E27AB515F233F
:1009C000AC516023AD516123AE515E27AF515F231F
:1009D000B0516023B1516123B2515E27B3515F23FF
:1009E000B4516023B5516123B6515E27B7515F23DF
:1009F000B8516023B9516123D8900101613360334C
:100A00005F335E33D8900101613360335F335E330F
:100A1000D8900101613360335F335E3300C10CF164
:100A200001C10DF102C10EF103C10FF104C110F1BA
:100A300005C111F106C112F107C113F108C114F18A
:100A400009C115F10AC116F10BC117F134C135F115
:100A500011B836EF05F00101620E046F010E056F4B
:100A6000000E066F000E076F3FEF05F00101A70EA5
:100A7000046F020E056F000E066F000E076F5EC159
:100A800000F15FC101F160C102F161C103F1DAEC73
:100A90002CF003BF04D019BE02D019A0108C11A0F5
:100AA00057EF05F010BA57EF05F00F80108A0CC110
:100AB00000F10DC101F10EC102F10FC103F110C12E
:100AC00004F111C105F112C106F113C107F114C1FE
:100AD00008F115C109F116C10AF117C10BF135C1B1
:100AE00034F113EF0BF00392ABB2AB98AB88030178
:100AF00003EE00F080517F0BE92604C0EFFF802B4E
:100B00008151805D700BD8A48B8200008051815D83
:100B1000700BD8A48B9281518019D8B4079013EF31
:100B20000BF0F2940101453F13EF0BF0462B13EF4E
:100B30000BF09E900101533F13EF0BF0542B13EF7A
:100B40000BF09E9211B82BEF08F0040066A1A9EFFC
:100B500005F08BB4B3EF05F010ACB3EF05F08B8468
:100B6000109CB4EF05F08B94077C07ACCFEF05F039
:100B7000C274C2B4C9EF05F0C3CFB7F5C4CFB8F59E
:100B80000501D890B833B733D890B833B733D0EF26
:100B900005F0C3CF55F1C4CF56F1D0EF05F0C282B6
:100BA00007B442EF06F047C14BF148C14CF149C1CF
:100BB0004DF14AC14EF15EC162F15FC163F160C1A6
:100BC00064F161C165F113A8E8EF05F0138C139887
:100BD0009AC1BAF19BC1BBF19CC1BCF19DC1BDF1F1
:100BE0009EC1BEF19FC1BFF1A0C1C0F1A1C1C1F1C1
:100BF000A2C1C2F1A3C1C3F1A4C1C4F1A5C1C5F191
:100C0000A6C1C6F1A7C1C7F1A8C1C8F1A9C1C9F160
:100C1000AAC1CAF1ABC1CBF1ACC1CCF1ADC1CDF130
:100C2000AEC1CEF1AFC1CFF1B0C1D0F1B1C1D1F100
:100C3000B2C1D2F1B3C1D3F1B4C1D4F1B5C1D5F1D0
:100C4000B6C1D6F1B7C1D7F1B8C1D8F1B9C1D9F1A0
:100C5000B7C5B9F5B8C5BAF5B9C5BBF5BAC5BCF5E0
:100C6000010155515B2756515C23E86A5D230E2E26
:100C700042EF06F05CC157F15DC158F15B6B5C6BF4
:100C80005D6B078E0201002F13EF0BF03C0E006F1F
:100C90001A50E00BE00AE866128818BE02D018B4B9
:100CA000108E00C10CF101C10DF102C10EF103C1A2
:100CB0000FF104C110F105C111F106C112F107C114
:100CC00013F108C114F109C115F10AC116F10BC1E4
:100CD00017F134C135F181AA23EF07F030A0F3EF0B
:100CE00006F005012F51000AD8B423EF07F00501E3
:100CF0002F51010AD8B4ACEF06F005012F51020ABA
:100D0000D8B4EDEF06F005012F51030AD8B4EDEF8A
:100D100006F005012F51040AD8B4EDEF06F00501E5
:100D20002F51050AD8B4EDEF06F005012F51060A40
:100D3000D8B4EDEF06F005012F51070AD8B4EDEF56
:100D400006F005012F51320AD8B4AAEF06F02F6B36
:100D500023EF07F023EF07F005015767B7EF06F021
:100D60005867B7EF06F05967B7EF06F05A67BBEF61
:100D700006F023EF07F05BC500F15CC501F15DC52E
:100D800002F15EC503F10101010E046F000E056F53
:100D9000000E066F000E076FDAEC2CF000C15BF559
:100DA00001C15CF502C15DF503C15EF50067E0EFCE
:100DB00006F00167E0EF06F00267E0EF06F0036778
:100DC00023EF07F057C55BF558C55CF559C55DF5D0
:100DD0005AC55EF50F8823EF07F005013067F3EF82
:100DE00006F023EF07F00FBE08EF07F010A00DEF9D
:100DF00007F00101476704EF07F0486704EF07F0C9
:100E0000496704EF07F04A6708EF07F00DEF07F0B6
:100E100007AE0DEF07F020EF07F00501312F23EFAC
:100E200007F03C0E316F302F23EF07F00101000E69
:100E3000626FE00E636FA50E646F010E656F13881D
:100E40000501306B0F880501666B37B729EF07F096
:100E500066810CC100F10DC101F10EC102F10FC19B
:100E600003F110C104F111C105F112C106F113C162
:100E700007F114C108F115C109F116C10AF117C132
:100E80000BF135C134F100C10CF101C10DF102C10A
:100E90000EF103C10FF104C110F105C111F106C13A
:100EA00012F107C113F108C114F109C115F10AC10A
:100EB00016F10BC117F134C135F101018E6768EFEE
:100EC00007F08F6768EF07F0906768EF07F09167AA
:100ED0006CEF07F09CEF07F092C100F193C101F1B4
:100EE00094C102F195C103F10101010E046F000EDE
:100EF000056F000E066F000E076FDAEC2CF000C1D4
:100F000092F101C193F102C194F103C195F100671F
:100F100091EF07F0016791EF07F0026791EF07F09B
:100F200003679CEF07F08EC192F18FC193F190C1DE
:100F300094F191C195F10F80D57ED5BE6ED0D6CFFC
:100F400047F1D7CF48F145C149F1E86AE8CF4AF106
:100F5000138A19BE02D019A0108C109047C100F15D
:100F600048C101F149C102F14AC103F101010A0E70
:100F7000046F000E056F000E066F000E076FDAECAF
:100F80002CF003AF1080010154A7D3EF07F00F9AA4
:100F90000F9C0F9E0101000E5E6F600E5F6F3D0E95
:100FA000606F080E616F010147BFE3EF07F048670C
:100FB000E3EF07F04967E3EF07F04A67E3EF07F075
:100FC000F28808EF08F0F2985E6B5F6B606B616B04
:100FD0009A6B9B6B9C6B9D6B9E6B9F6BA06BA16BCD
:100FE000A26BA36BA46BA56BA66BA76BA86BA96B7D
:100FF000AA6BAB6BAC6BAD6BAE6BAF6BB06BB16B2D
:10100000B26BB36BB46BB56BB66BB76BB86BB96BDC
:10101000D76AD66A0101456B466B0CC100F10DC160
:1010200001F10EC102F10FC103F110C104F111C1B0
:1010300005F112C106F113C107F114C108F115C180
:1010400009F116C10AF117C10BF135C134F113EFE3
:101050000BF013EF0BF00201002F77EF0AF0D59E93
:10106000D6CF47F1D7CF48F145C149F1E86AE8CF7B
:101070004AF1138AD76AD66A0101456B466BD58E51
:101080001A50E00BE00AE866128818BE02D018B4C5
:10109000108E17AE1C8C00C10CF101C10DF102C104
:1010A0000EF103C10FF104C110F105C111F106C128
:1010B00012F107C113F108C114F109C115F10AC1F8
:1010C00016F10BC117F134C135F10FA0109A11B808
:1010D00075EF08F00101620E046F010E056F000E3E
:1010E000066F000E076F7EEF08F00101A70E046F78
:1010F000020E056F000E066F000E076F47C100F16C
:1011000048C101F149C102F14AC103F1DAEC2CF006
:1011100003BF91EF08F019BE02D019A0108C11B0D6
:101120000F800CC100F10DC101F10EC102F10FC120
:1011300003F110C104F111C105F112C106F113C18F
:1011400007F114C108F115C109F116C10AF117C15F
:101150000BF135C134F102013C0E006F00C10CF1FE
:1011600001C10DF102C10EF103C10FF104C110F173
:1011700005C111F106C112F107C113F108C114F143
:1011800009C115F10AC116F10BC117F134C135F1CE
:1011900081AA80EF09F030A050EF09F005012F512E
:1011A000000AD8B480EF09F005012F51010AD8B424
:1011B00009EF09F005012F51020AD8B44AEF09F0EE
:1011C00005012F51030AD8B44AEF09F005012F5148
:1011D000040AD8B44AEF09F005012F51050AD8B422
:1011E0004AEF09F005012F51060AD8B44AEF09F079
:1011F00005012F51070AD8B44AEF09F005012F5114
:10120000320AD8B407EF09F02F6B80EF09F080EFB6
:1012100009F00501576714EF09F0586714EF09F05A
:10122000596714EF09F05A6718EF09F080EF09F0D9
:101230005BC500F15CC501F15DC502F15EC503F15E
:101240000101010E046F000E056F000E066F000E07
:10125000076FDAEC2CF000C15BF501C15CF502C14F
:101260005DF503C15EF500673DEF09F001673DEFF5
:1012700009F002673DEF09F0036780EF09F057C5F9
:101280005BF558C55CF559C55DF55AC55EF50F8827
:1012900080EF09F00501306750EF09F080EF09F0A9
:1012A0000FBE65EF09F010A06AEF09F00101476772
:1012B00061EF09F0486761EF09F0496761EF09F0F4
:1012C0004A6765EF09F06AEF09F007AE6AEF09F0C7
:1012D0007DEF09F00501312F80EF09F03C0E316FF1
:1012E000302F80EF09F00101000E626FE00E636F96
:1012F000A50E646F010E656F13880501306B0F88B2
:101300000501666B37B786EF09F066810CC100F105
:101310000DC101F10EC102F10FC103F110C104F1C1
:1013200011C105F112C106F113C107F114C108F191
:1013300015C109F116C10AF117C10BF135C134F11C
:1013400000C10CF101C10DF102C10EF103C10FF199
:1013500004C110F105C111F106C112F107C113F169
:1013600008C114F109C115F10AC116F10BC117F139
:1013700034C135F101018E67C5EF09F08F67C5EF04
:1013800009F09067C5EF09F09167C9EF09F0F9EF2F
:1013900009F092C100F193C101F194C102F195C12C
:1013A00003F10101010E046F000E056F000E066FC0
:1013B000000E076FDAEC2CF000C192F101C193F13D
:1013C00002C194F103C195F10067EEEF09F00167E6
:1013D000EEEF09F00267EEEF09F00367F9EF09F0AD
:1013E0008EC192F18FC193F190C194F191C195F1A9
:1013F0000F80109047C100F148C101F149C102F1CD
:101400004AC103F101010A0E046F000E056F000EC0
:10141000066F000E076FDAEC2CF003AF10800101AD
:1014200054A71FEF0AF00F9A0F9C0F9E0101000EA8
:101430005E6F600E5F6F3D0E606F080E616F47C19B
:1014400000F148C101F149C102F14AC103F10101B2
:10145000140E046F050E056F000E066F000E076F69
:10146000DAEC2CF003AF38EF0AF0F2885DEF0AF007
:10147000F2985E6B5F6B606B616B9A6B9B6B9C6BA6
:101480009D6B9E6B9F6BA06BA16BA26BA36BA46B00
:10149000A56BA66BA76BA86BA96BAA6BAB6BAC6BB0
:1014A000AD6BAE6BAF6BB06BB16BB26BB36BB46B60
:1014B000B56BB66BB76BB86BB96B0CC100F10DC1F6
:1014C00001F10EC102F10FC103F110C104F111C10C
:1014D00005F112C106F113C107F114C108F115C1DC
:1014E00009F116C10AF117C10BF135C134F104003D
:1014F0008BB482EF0AF010AC82EF0AF08B84109C60
:1015000083EF0AF08B94077C07AC9EEF0AF0C2745D
:10151000C2B498EF0AF0C3CFB7F5C4CFB8F5050150
:10152000D890B833B733D890B833B7339FEF0AF0B9
:10153000C3CF55F1C4CF56F19FEF0AF0C28207B472
:1015400011EF0BF047C14BF148C14CF149C14DF1CE
:101550004AC14EF15EC162F15FC163F160C164F1E5
:1015600061C165F113A8B7EF0AF0138C13989AC103
:10157000BAF19BC1BBF19CC1BCF19DC1BDF19EC143
:10158000BEF19FC1BFF1A0C1C0F1A1C1C1F1A2C113
:10159000C2F1A3C1C3F1A4C1C4F1A5C1C5F1A6C1E3
:1015A000C6F1A7C1C7F1A8C1C8F1A9C1C9F1AAC1B3
:1015B000CAF1ABC1CBF1ACC1CCF1ADC1CDF1AEC183
:1015C000CEF1AFC1CFF1B0C1D0F1B1C1D1F1B2C153
:1015D000D2F1B3C1D3F1B4C1D4F1B5C1D5F1B6C123
:1015E000D6F1B7C1D7F1B8C1D8F1B9C1D9F1B7C5F2
:1015F000B9F5B8C5BAF5B9C5BBF5BAC5BCF50101B1
:1016000055515B2756515C23E86A5D230E2E11EF7E
:101610000BF05CC157F15DC158F15B6B5C6B5D6BAE
:10162000078E13EF0BF002C0E0FF005001C0D8FF9F
:101630001000A6B219EF0BF00CC0A9FF0BC0A8FF59
:10164000A69EA69CA684F29E550EA76EAA0EA76E15
:10165000A682F28EA694A6B22BEF0BF00C2A1200F3
:10166000A96EA69EA69CA680A8500C2A1200040172
:101670002C0E826F82EC0EF0D5EC2DF00C5030EC7D
:101680000BF0E8CF00F10C5030EC0BF0E8CF01F19B
:1016900001AF50EF0BF00101FF0E026FFF0E036F61
:1016A00078EC2DF029675CEF0BF00401200E826FBF
:1016B00082EC0EF061EF0BF004012D0E826F82ECD4
:1016C0000EF082EC2BF01200306A076A0F6A106A83
:1016D000116A126A136A0F010D0EC16E860EC06E7A
:1016E000030EC26E0F01680E896E130E926E080E05
:1016F0008A6EF30E936E8B6A900E946EC80E30EC69
:101700000BF0E8CFE8FF1098E8A0108810A805D0EB
:101710000E0E226E8E0E236E04D00F0E226E8F0ED2
:10172000236E54EC2EF0F18EF19EFC0E30EC0BF09B
:10173000E8CF0BF00BA011800BA211820BA4118437
:101740000BA81188C90E30EC0BF0E8CF17F0CA0EC9
:1017500030EC0BF0E8CF18F0CB0E30EC0BF0E8CF0C
:1017600019F0CC0E30EC0BF0E8CF1AF0CD0E30ECC7
:101770000BF0E8CF2FF01C6A1D6A0E6A01015B6B4B
:101780005C6B5D6B576B586BF29A0101476B486B52
:10179000496B4A6B4B6B4C6B4D6B4E6B4F6B506B8D
:1017A000516B526B456B466BD76AD66A0F01280E98
:1017B000D56EF28A9D90B00ECD6E01015E6B5F6BAF
:1017C000606B616B626B636B646B656B666B676BA5
:1017D000686B696B536B546BCF6ACE6A0F9A0F9C20
:1017E0000F9E9D80760ECA6E9D8202013C0E006F98
:1017F000CC6A160E30EC0BF0E8CF00F1170E30EC8F
:101800000BF0E8CF01F1180E30EC0BF0E8CF02F14D
:10181000190E30EC0BF0E8CF03F1010103AF2BEF11
:101820000CF0D5EC2DF0160E0C6E00C10BF019EC7F
:101830000BF0170E0C6E01C10BF019EC0BF0180E2B
:101840000C6E02C10BF019EC0BF0190E0C6E03C1FB
:101850000BF019EC0BF000C18EF101C18FF102C148
:1018600090F103C191F100C192F101C193F102C164
:1018700094F103C195F11A0E30EC0BF0E8CF00F1B2
:101880001B0E30EC0BF0E8CF01F11C0E30EC0BF02E
:10189000E8CF02F11D0E30EC0BF0E8CF03F10101AF
:1018A00003AF81EF0CF0D5EC2DF01A0E0C6E00C1D9
:1018B0000BF019EC0BF01B0E0C6E01C10BF019ECC8
:1018C0000BF01C0E0C6E02C10BF019EC0BF01D0E90
:1018D0000C6E03C10BF019EC0BF01A0E30EC0BF090
:1018E000E8CF00F11B0E30EC0BF0E8CF01F11C0E3D
:1018F00030EC0BF0E8CF02F11D0E30EC0BF0E8CF2E
:1019000003F100C196F101C197F102C198F103C141
:1019100099F1240EAC6E900EAB6E240EAC6E080ED8
:10192000B86E000EB06E1F0EAF6E0401806B816B3F
:101930000F01900EAB6E0F019D8A0301806B816BCE
:10194000C26B8B92F8EC32F0F8EC32F056EC34F0DB
:10195000D7EC30F0200E30EC0BF0E8CF2FF505017E
:101960002F51FF0AD8A4BCEF0CF02F6B200E0C6E89
:101970002FC50BF019EC0BF00501010E306F3C0E7A
:10198000316F250E30EC0BF0E8CF00F1260E30EC75
:101990000BF0E8CF01F1270E30EC0BF0E8CF02F1AD
:1019A000280E30EC0BF0E8CF03F1010103AFF3EFA9
:1019B0000CF0D5EC2DF0250E0C6E00C10BF019ECDF
:1019C0000BF0260E0C6E01C10BF019EC0BF0270E7C
:1019D0000C6E02C10BF019EC0BF0280E0C6E03C15B
:1019E0000BF019EC0BF000C157F501C158F502C11D
:1019F00059F503C15AF500C15BF501C15CF502C19F
:101A00005DF503C15EF5290E30EC0BF0E8CF5FF514
:101A1000050160515F5DD8A05FC560F5210E30EC17
:101A20000BF0E8CF00F1220E30EC0BF0E8CF01F123
:101A3000230E30EC0BF0E8CF02F1240E30EC0BF06B
:101A4000E8CF03F1010103AF54EF0DF0D5EC2DF019
:101A5000210E0C6E00C10BF019EC0BF0220E0C6E77
:101A600001C10BF019EC0BF0230E0C6E02C10BF050
:101A700019EC0BF0240E0C6E03C10BF019EC0BF0FB
:101A8000210E30EC0BF0E8CF00F1220E30EC0BF021
:101A9000E8CF01F1230E30EC0BF0E8CF02F1240E79
:101AA00030EC0BF0E8CF03F100C161F501C162F544
:101AB00002C163F503C164F51FEC30F005EC2FF0B3
:101AC0005DEC2EF030A0C5EF0DF005012F51020A9C
:101AD00016E005012F51030A19E005012F51040AF0
:101AE00024E005012F51050A2BE005012F51060ABC
:101AF00039E005012F51070A3FE0C5EF0DF0602FD7
:101B0000C2EF0DF05FC560F5C5EF0DF0B0C500F197
:101B100001010F0E001701010051000A36E001011A
:101B20000051050A32E0C2EF0DF0B0C500F101012D
:101B30000F0E001701010051000A27E0C2EF0DF05F
:101B40000501B051000A21E00501B051150A1DE060
:101B50000501B051300A19E00501B051450A15E000
:101B6000C2EF0DF00501B051000A0FE00501B051C0
:101B7000300A0BE0C2EF0DF00501B051000A05E09C
:101B8000C2EF0DF081BA95EF34F007900001F28EAC
:101B9000F28C12AE03D012BCC1EF18F007B008EF00
:101BA0002AF00FB01BEF23F010BE1BEF23F012B88A
:101BB0001BEF23F00FB8A9EF1CF00301805181192E
:101BC0007F0BD8B408EF2AF013EE00F081517F0BA1
:101BD000E126812BE7CFE8FFE00BD8B408EF2AF02D
:101BE00023EE82F0C2513F0BD926E7CFDFFFC22B95
:101BF000DF50780AD8A408EF2AF0078092C100F1DC
:101C000093C101F194C102F195C103F10101040EE8
:101C1000046F000E056F000E066F000E076FDAEC02
:101C20002CF000AF1DEF0EF00101030E926F000EBD
:101C3000936F000E946F000E956F03018251720A2C
:101C4000D8B4F7EF22F08251520AD8B4F7EF22F05D
:101C50008251750AD8B4F7EF22F08251630AD8B4E2
:101C6000C2EF26F08251690AD8B4A1EF1FF0825169
:101C70007A0AD8B4B4EF20F08251490AD8B440EFC0
:101C80001FF08251500AD8B45EEF1EF08251700AE4
:101C9000D8B4A1EF1EF08251540AD8B4CCEF1EF094
:101CA0008251740AD8B412EF1FF08251410AD8B49D
:101CB00098EF0FF082514B0AD8B496EF0EF0825194
:101CC0006D0AD8B4CBEF13F082514D0AD8B4E4EFCB
:101CD00013F08251730AD8B427EF22F08251530ACD
:101CE000D8B48CEF22F082514C0AD8B473EF14F0C0
:101CF0008251590AD8B41CEF13F012AE01D0128CE5
:101D0000F9EF26F0040114EE00F080517F0BE1267C
:101D100082C4E7FF802B120004010D0E826F82EC5B
:101D20000EF00A0E826F82EC0EF0120004014B0ED0
:101D3000826F82EC0EF004012C0E826F82EC0EF0AA
:101D400081B802D02FB630D003018351430AD8B4F2
:101D5000DBEF0EF003018351630AD8B4DDEF0EF020
:101D600003018351520AD8B4DFEF0EF0030183510F
:101D7000720AD8B4E1EF0EF003018351470AD8B4D8
:101D8000E3EF0EF003018351670AD8B4E5EF0EF0DC
:101D900003018351540AD8B4E7EF0EF003018351D5
:101DA000740AD8B456EF0FF003018351550AD8B422
:101DB000E9EF0EF082D02F807AD02F9078D02F824A
:101DC00076D02F9274D02F8472D02F9470D02F861B
:101DD0006ED084C330F185C331F186C332F187C33D
:101DE00033F10101296B23EC2EF09AEC2DF000C1A8
:101DF00004F101C105F102C106F103C107F116ECBE
:101E00002EF0200EF86EF76AF66A0900F5CF2CF175
:101E10000900F5CF2DF10900F5CF2EF10900F5CF1E
:101E20002FF10900F5CF30F10900F5CF31F10900AC
:101E3000F5CF32F10900F5CF33F10101296B23EC25
:101E40002EF09AEC2DF0DAEC2CF000672FEF0FF06B
:101E500001672FEF0FF002672FEF0FF0036701D03C
:101E600025D004014E0E826F82EC0EF004016F0E3D
:101E7000826F82EC0EF004014D0E826F82EC0EF048
:101E80000401610E826F82EC0EF00401740E826F09
:101E900082EC0EF00401630E826F82EC0EF00401FE
:101EA000680E826F82EC0EF0F7EF26F02F96CD0EC3
:101EB0000C6E2FC00BF019EC0BF0CD0E30EC0BF0CC
:101EC000E8CF2FF02FB006D00401630E826F82ECB2
:101ED0000EF005D00401430E826F82EC0EF02FB29B
:101EE00006D00401720E826F82EC0EF005D0040160
:101EF000520E826F82EC0EF02FB406D00401670EF2
:101F0000826F82EC0EF005D00401470E826F82ECE6
:101F10000EF02FB606D00401740E826F82EC0EF024
:101F200005D00401540E826F82EC0EF0F7EF26F01C
:101F30000401410E826F82EC0EF003018351310ADD
:101F4000D8B43CEF12F003018351320AD8B46CEFDD
:101F500011F003018351330AD8B4F5EF10F00301F7
:101F60008351340AD8B4E5EF0FF003018351350AE9
:101F7000D8B4C2EF0FF004013F0E826F82EC0EF076
:101F8000F7EF26F004012C0E826F82EC0EF00301B5
:101F90008451300AD8B4D5EF0FF003018451310ACF
:101FA000D8B4DDEF0FF02EEF11F08B900401300E5E
:101FB000826F82EC0EF0E3EF0FF08B800401310EA4
:101FC000826F82EC0EF0F7EF26F0CC0E30EC0BF0C7
:101FD000E8CF0BF004012C0E826F82EC0EF00301AF
:101FE0008451310AD8B409EF10F003018451300A4A
:101FF000D8B40BEF10F0030184514D0AD8B415EF9B
:1020000010F003018451540AD8B41CEF10F033EFE0
:1020100010F08A8401D08A940BAE04D00BAC02D0AD
:102020000BBA21D0E00E0B1218D01F0E0B168539FB
:10203000E844E00B0B1211D0E00E0B1616EC2EF05C
:1020400085C332F186C333F10101296B23EC2EF0F5
:102050009AEC2DF000511F0B0B12CC0E0C6E0BC026
:102060000BF019EC0BF00401340E826F82EC0EF0D1
:1020700004012C0E826F82EC0EF0CC0E30EC0BF0D3
:10208000E8CF1AF08AB406D00401300E826F82ECD9
:102090000EF005D00401310E826F82EC0EF00401C7
:1020A0002C0E826F82EC0EF01A38E840070BE8CF56
:1020B00082F40401300E822782EC0EF004012C0E13
:1020C000826F82EC0EF0D5EC2DF01A501F0BE8CF8A
:1020D00000F178EC2DF032C182F40401300E822739
:1020E00082EC0EF033C182F40401300E822782ECC0
:1020F0000EF004012C0E826F82EC0EF0D5EC2DF068
:102100002DC000F100AF0BD0FF0E016FFF0E026F6C
:10211000FF0E036F04012D0E826F82EC0EF078EC3F
:102120002DF031C182F40401300E822782EC0EF0D2
:1021300032C182F40401300E822782EC0EF033C1EA
:1021400082F40401300E822782EC0EF004012C0E82
:10215000826F82EC0EF0D5EC2DF02CC000F178EC03
:102160002DF031C182F40401300E822782EC0EF092
:1021700032C182F40401300E822782EC0EF033C1AA
:1021800082F40401300E822782EC0EF004012C0E42
:10219000826F82EC0EF0D5EC2DF02EC000F100AF76
:1021A0000BD0FF0E016FFF0E026FFF0E036F0401D5
:1021B0002D0E826F82EC0EF078EC2DF031C182F49E
:1021C0000401300E822782EC0EF032C182F4040149
:1021D000300E822782EC0EF033C182F40401300EFF
:1021E000822782EC0EF0F7EF26F0CB0E30EC0BF0EE
:1021F000E8CF0BF004012C0E826F82EC0EF003018D
:102200008451450AD8B419EF11F003018451440AEE
:10221000D8B41CEF11F003018451300AD8B41FEF79
:1022200011F003018451310AD8B423EF11F02EEFDD
:1022300011F00B9E28EF11F00B8E28EF11F0FC0E21
:102240000B1628EF11F0FC0E0B160B8028EF11F087
:10225000CB0E0C6E0BC00BF019EC0BF00401330E1F
:10226000826F82EC0EF004012C0E826F82EC0EF075
:10227000CB0E30EC0BF0E8CF19F019BE47EF11F0A0
:102280000401450E826F82EC0EF04CEF11F0040158
:10229000440E826F82EC0EF004012C0E826F82ECF1
:1022A0000EF00401300E826F82EC0EF004012C0E51
:1022B000826F82EC0EF019B065EF11F00401300E60
:1022C000826F82EC0EF06AEF11F00401310E826F22
:1022D00082EC0EF0F7EF26F0CA0E30EC0BF0E8CFF0
:1022E0000BF004012C0E826F82EC0EF0030184517E
:1022F000450AD8B4A8EF11F003018451440AD8B4B8
:10230000ABEF11F0030184514D0AD8B4B4EF11F0D2
:1023100003018451410AD8B4AEEF11F00301845196
:10232000460AD8B4B1EF11F003018451560AD8B46B
:10233000BCEF11F003018451500AD8B4C7EF11F07B
:1023400003018451520AD8B4CAEF11F0D3EF11F04F
:102350000B9ECDEF11F00B8ECDEF11F00B9CCDEF5E
:1023600011F00B8CCDEF11F0FC0E0B1685C3E8FFBE
:10237000030B0B12CDEF11F0C70E0B1685C3E8FF50
:10238000070BE846E846E8460B12CDEF11F00B8448
:10239000CDEF11F00B94CDEF11F0CA0E0C6E0BC007
:1023A0000BF019EC0BF0CA0E30EC0BF0E8CF18F084
:1023B0000401320E826F82EC0EF004012C0E826F4B
:1023C00082EC0EF018BEECEF11F00401450E826FA6
:1023D00082EC0EF0F1EF11F00401440E826F82ECFA
:1023E0000EF004012C0E826F82EC0EF018C0E8FF94
:1023F000030BE8CF82F40401300E822782EC0EF04A
:1024000004012C0E826F82EC0EF018BC0FEF12F05C
:102410000401410E826F82EC0EF014EF12F0040101
:10242000460E826F82EC0EF004012C0E826F82EC5D
:102430000EF018C0E8FF380BE842E842E842E8CF67
:1024400082F40401300E822782EC0EF004012C0E7F
:10245000826F82EC0EF018B435EF12F00401520EC8
:10246000826F82EC0EF03AEF12F00401500E826F90
:1024700082EC0EF0F7EF26F0C90E30EC0BF0E8CF4F
:102480000BF004012C0E826F82EC0EF003018451DC
:10249000450AD8B45AEF12F003018451440AD8B463
:1024A0005DEF12F0030184514D0AD8B460EF12F0D1
:1024B0006EEF12F00B9E68EF12F00B8E68EF12F0C9
:1024C000F80E0B1685C3E8FF070B0B1268EF12F02E
:1024D000C90E0C6E0BC00BF019EC0BF00401310EA1
:1024E000826F82EC0EF004012C0E826F82EC0EF0F3
:1024F000C90E30EC0BF0E8CF17F017BE06D0040180
:10250000450E826F82EC0EF005D00401440E826FFE
:1025100082EC0EF004012C0E826F82EC0EF017C0DC
:10252000E8FF070BE8CF82F40401300E822782EC2B
:102530000EF004012C0E826F82EC0EF00780D5ECB9
:102540002DF028C0E8FF003B00430043030B78EC6C
:102550002DF033C182F40401300E822782EC0EF09C
:1025600004012C0E826F82EC0EF0D5EC2DF028C009
:1025700001F1019F019D29C000F1010178EC2DF0CE
:102580002FC182F40401300E822782EC0EF030C19C
:1025900082F40401300E822782EC0EF031C182F405
:1025A0000401300E822782EC0EF032C182F4040165
:1025B000300E822782EC0EF033C182F40401300E1B
:1025C000822782EC0EF004012C0E826F82EC0EF05A
:1025D000D5EC2DF02AC001F12BC000F1D8900133C9
:1025E0000033D89001330033010178EC2DF02FC176
:1025F00082F40401300E822782EC0EF030C182F4A6
:102600000401300E822782EC0EF031C182F4040105
:10261000300E822782EC0EF032C182F40401300EBB
:10262000822782EC0EF033C182F40401300E82273F
:1026300082EC0EF0F7EF26F0FC0E30EC0BF0E8CF5A
:102640000BF003018351520AD8B453EF13F0030186
:102650008351720AD8B456EF13F003018351500A24
:10266000D8B459EF13F003018351700AD8B45CEF6A
:1026700013F003018351550AD8B45FEF13F003013F
:102680008351750AD8B462EF13F003018351430AF2
:10269000D8B46BEF13F003018351630AD8B46EEF23
:1026A00013F077EF13F00B9071EF13F00B8071EFD5
:1026B00013F00B9271EF13F00B8271EF13F00B9488
:1026C00071EF13F00B8471EF13F00B9671EF13F0B1
:1026D0000B8671EF13F00B9871EF13F00B8871EF0D
:1026E00013F0FC0E0C6E0BC00BF019EC0BF0040198
:1026F000590E826F82EC0EF0119011921194119884
:10270000FC0E30EC0BF0E8CF0BF00BA011800BA20D
:1027100011820BA411840BA8118811A097EF13F05C
:102720000401520E826F82EC0EF09CEF13F0040154
:10273000720E826F82EC0EF011A8A6EF13F0040166
:10274000430E826F82EC0EF0ABEF13F00401630EC8
:10275000826F82EC0EF011A2B5EF13F00401500E5F
:10276000826F82EC0EF0BAEF13F00401700E826FEC
:1027700082EC0EF011A4C4EF13F00401550E826F29
:1027800082EC0EF0C9EF13F00401750E826F82EC3B
:102790000EF0F7EF26F004016D0E826F82EC0EF062
:1027A00003018351300AD8B423EF14F0030183519D
:1027B000310AD8B436EF14F003018351320AD8B489
:1027C00049EF14F0F9EF26F004014D0E826F82EC10
:1027D0000EF016EC2EF084C331F185C332F186C3BE
:1027E00033F10101296B23EC2EF09AEC2DF003015B
:1027F0008351300AD8B40BEF14F003018351310A2E
:10280000D8B413EF14F003018351320AD8B41BEF8C
:1028100014F0F9EF26F0FD0E0C6E00C10BF019EC70
:102820000BF023EF14F0FE0E0C6E00C10BF019EC50
:102830000BF036EF14F0FF0E0C6E00C10BF019EC2C
:102840000BF049EF14F00401300E826F82EC0EF0B1
:1028500004012C0E826F82EC0EF0D5EC2DF0FD0EF3
:1028600030EC0BF0E8CF00F15AEF14F00401310E18
:10287000826F82EC0EF004012C0E826F82EC0EF05F
:10288000D5EC2DF0FE0E30EC0BF0E8CF00F15AEF56
:1028900014F00401320E826F82EC0EF0D5EC2DF0B4
:1028A00004012C0E826F82EC0EF0FF0E30EC0BF068
:1028B000E8CF00F178EC2DF031C182F40401300E44
:1028C000822782EC0EF032C182F40401300E82279E
:1028D00082EC0EF033C182F40401300E822782ECC8
:1028E0000EF0F7EF26F003018351300AD8B46EEFF3
:1028F00019F003018351310AD8B49BEF1AF0030198
:102900008351320AD8B409EF1BF003018351330A13
:10291000D8B419EF1BF003018351340AD8B429EF5E
:102920001BF003018351350AD8B4AFEF1CF003014B
:102930008351360AD8B4DDEF1CF003018351370A06
:10294000D8B446EF17F003018351380AD8B4E4EF46
:1029500017F003018351460AD8B402EF1CF00301BB
:1029600083514D0AD8B4BFEF15F0030183516D0AAE
:10297000D8B4D9EF15F0030183515A0AD8B415EF32
:102980001AF003018351490AD8B4DDEF1DF00301A9
:102990008351500AD8B40FEF1DF003018351540A3C
:1029A000D8B488EF1DF003018351630AD8B4F9EF5E
:1029B00015F003018351430AD8B4F1EF16F0030177
:1029C0008351730AD8B4F7EF15F003018351610AFC
:1029D000D8B40CEF15F003018351650AD8B4BEEFEB
:1029E00019F003018351450AD8B4CCEF19F0030163
:1029F0008351620AD8B4DAEF19F003018351420A15
:102A0000D8B4E8EF19F003018351760AD8B4F6EF91
:102A100019F0D8A4F9EF26F004014C0E826F82EC75
:102A20000EF00401610E826F82EC0EF005EC2FF0C7
:102A300004012C0E826F82EC0EF0D5EC2DF0AFC5A8
:102A400000F1010178EC2DF031C182F40401300E67
:102A5000822782EC0EF032C182F40401300E82270C
:102A600082EC0EF033C182F40401300E822782EC36
:102A70000EF004012C0E826F82EC0EF0D5EC2DF0DE
:102A8000B0C500F1010178EC2DF031C182F40401F0
:102A9000300E822782EC0EF032C182F40401300E37
:102AA000822782EC0EF033C182F40401300E8227BB
:102AB00082EC0EF004012C0E826F82EC0EF0D5EC4D
:102AC0002DF0B1C500F1010178EC2DF031C182F497
:102AD0000401300E822782EC0EF032C182F4040130
:102AE000300E822782EC0EF033C182F40401300EE6
:102AF000822782EC0EF004012C0E826F82EC0EF025
:102B0000D5EC2DF0B2C500F1010178EC2DF031C10A
:102B100082F40401300E822782EC0EF032C182F47E
:102B20000401300E822782EC0EF033C182F40401DE
:102B3000300E822782EC0EF004012C0E826F82ECA4
:102B40000EF0D5EC2DF0B6C500F1010178EC2DF0BA
:102B500031C182F40401300E822782EC0EF032C1C2
:102B600082F40401300E822782EC0EF033C182F42D
:102B70000401300E822782EC0EF00BEF1DF016ECF4
:102B80002EF084C333F123EC2EF09AEC2DF0200EBE
:102B90000C6E00C10BF019EC0BF000C12FF5050114
:102BA0002F51000A06E005012F51010A02E09FECB7
:102BB0002FF004014C0E826F82EC0EF004014D0EDA
:102BC000826F82EC0EF004012C0E826F82EC0EF00C
:102BD000D5EC2DF02FC500F178EC2DF033C182F447
:102BE0000401300E822782EC0EF00BEF1DF095EF02
:102BF00034F004014C0E826F82EC0EF00401630E7F
:102C0000826F82EC0EF05DEC2EF004012C0E826FD0
:102C100082EC0EF00EEC16F00BEF1DF0D5EC2DF063
:102C2000B5C500F10101003B0F0E001778EC2DF047
:102C300033C182F40401300E822782EC0EF0B5C558
:102C400000F101010F0E0101001778EC2DF033C1E6
:102C500082F40401300E822782EC0EF004012D0E66
:102C6000826F82EC0EF0B4C500F10101003B0F0E43
:102C7000001778EC2DF033C182F40401300E822766
:102C800082EC0EF0B4C500F101010F0E0101001736
:102C900078EC2DF033C182F40401300E822782ECEF
:102CA0000EF004012D0E826F82EC0EF0B3C500F120
:102CB0000101003B0F0E001778EC2DF033C182F4B8
:102CC0000401300E822782EC0EF0B3C500F1010141
:102CD0000F0E0101001778EC2DF033C182F40401CE
:102CE000300E822782EC0EF00401200E826F82ECFF
:102CF0000EF0B2C500F10F0E0101001778EC2DF0B7
:102D000033C182F40401300E822782EC0EF00401FC
:102D1000200E826F82EC0EF0B1C500F101010101BD
:102D2000003B0F0E001778EC2DF033C182F4040144
:102D3000300E822782EC0EF0B1C500F101010F0EBA
:102D40000101001778EC2DF033C182F40401300E3C
:102D5000822782EC0EF004013A0E826F82EC0EF0B4
:102D6000B0C500F10101003B0F0E001778EC2DF00B
:102D700033C182F40401300E822782EC0EF0B0C51C
:102D800000F101010F0E0101001778EC2DF033C1A5
:102D900082F40401300E822782EC0EF004013A0E18
:102DA000826F82EC0EF0AFC500F10101003B0F0E07
:102DB000001778EC2DF033C182F40401300E822725
:102DC00082EC0EF0AFC500F101010F0E001778EC98
:102DD0002DF033C182F40401300E822782EC0EF014
:102DE000120084C3E8FF0F0BE83AE8CFB5F585C3BE
:102DF000E8FF0F0B0501B51387C3E8FF0F0BE83A97
:102E0000E8CFB4F588C3E8FF0F0B0501B4138AC3FC
:102E1000E8FF0F0BE83AE8CFB3F58BC3E8FF0F0BE1
:102E20000501B3138DC3E8FF0F0BE8CFB2F58FC3D5
:102E3000E8FF0F0BE83AE8CFB1F590C3E8FF0F0BBE
:102E40000501B11392C3E8FF0F0BE83AE8CFB0F5E4
:102E500093C3E8FF0F0B0501B01395C3E8FF0F0BF9
:102E6000E83AE8CFAFF596C3E8FF0F0B0501AF13C3
:102E7000B8EC2EF004014C0E826F82EC0EF00401CF
:102E8000430E826F82EC0EF003EF16F0078404010C
:102E90004C0E826F82EC0EF00401370E826F82ECD2
:102EA0000EF004012C0E826F82EC0EF005012E5103
:102EB000130A06E005012E51170A0DE0E1EF17F0A5
:102EC0000101000E006F000E016F100E026F000E68
:102ED000036F74EF17F00101000E006F000E016F19
:102EE000000E026F010E036F78EC2DF02AC182F400
:102EF0000401300E822782EC0EF02BC182F4040113
:102F0000300E822782EC0EF02CC182F40401300EC8
:102F1000822782EC0EF02DC182F40401300E82274C
:102F200082EC0EF02EC182F40401300E822782EC76
:102F30000EF02FC182F40401300E822782EC0EF0D5
:102F400030C182F40401300E822782EC0EF031C1D0
:102F500082F40401300E822782EC0EF032C182F43A
:102F60000401300E822782EC0EF033C182F404019A
:102F7000300E822782EC0EF004012C0E826F82EC60
:102F80000EF00101100E006F000E016F000E026FB7
:102F9000000E036F78EC2DF031C182F40401300E85
:102FA000822782EC0EF032C182F40401300E8227B7
:102FB00082EC0EF033C182F40401300E822782ECE1
:102FC0000EF007940BEF1DF00501216B226B236BB4
:102FD000246B04014C0E826F82EC0EF00401380E5B
:102FE000826F82EC0EF004012C0E826F82EC0EF0E8
:102FF0000101100E006F000E016F000E026F000E37
:10300000036F78EC2DF02AC182F40401300E822780
:1030100082EC0EF02BC182F40401300E822782EC88
:103020000EF02CC182F40401300E822782EC0EF0E7
:103030002DC182F40401300E822782EC0EF02EC1E5
:1030400082F40401300E822782EC0EF02FC182F44C
:103050000401300E822782EC0EF030C182F40401AC
:10306000300E822782EC0EF031C182F40401300E62
:10307000822782EC0EF032C182F40401300E8227E6
:1030800082EC0EF033C182F40401300E822782EC10
:103090000EF004012C0E826F82EC0EF025C500F1BB
:1030A00026C501F127C502F128C503F10101100E63
:1030B000046F000E056F000E066F000E076F0BEC1D
:1030C0002DF000C133F501C134F502C135F503C15E
:1030D00036F578EC2DF02AC182F40401300E8227F7
:1030E00082EC0EF02BC182F40401300E822782ECB8
:1030F0000EF02CC182F40401300E822782EC0EF017
:103100002DC182F40401300E822782EC0EF02EC114
:1031100082F40401300E822782EC0EF02FC182F47B
:103120000401300E822782EC0EF030C182F40401DB
:10313000300E822782EC0EF031C182F40401300E91
:10314000822782EC0EF032C182F40401300E822715
:1031500082EC0EF033C182F40401300E822782EC3F
:103160000EF08CEC0EF005013367BEEF18F03467FB
:10317000BEEF18F03567BEEF18F0366702D05DEF8E
:1031800019F0129E129C21C500F122C501F123C540
:1031900002F124C503F1899A400EC76E200EC66E57
:1031A0009E96C69E0B0EC96EFF0E9EB602D0E82EEE
:1031B000FCD79E96C69E02C1C9FFFF0E9EB602D0E6
:1031C000E82EFCD79E96C69E01C1C9FFFF0E9EB693
:1031D00002D0E82EFCD79E96C69E00C1C9FFFF0E06
:1031E0009EB602D0E82EFCD79E96C69EC952FF0E10
:1031F0009EB602D0E82EFCD70501100E326F0401F6
:1032000014EE00F080517F0BE1269E96C69EC952B7
:10321000FF0E9EB602D0E82EFCD7C9CFE7FF04010F
:10322000802B0501322FFFEF18F0898A33C500F19A
:1032300034C501F135C502F136C503F10101010EB6
:10324000046F000E056F000E066F000E076FDAECBC
:103250002CF000C133F501C134F502C135F503C1CD
:1032600036F5050133673CEF19F034673CEF19F090
:1032700035673CEF19F0366702D05DEF19F021C5D4
:1032800000F122C501F123C502F124C503F10101BA
:10329000100E046F000E056F000E066F000E076F14
:1032A000DFEC2CF000C121F501C122F502C123F5AC
:1032B00003C124F5128EF9EF26F00401450E826F4A
:1032C00082EC0EF004014F0E826F82EC0EF00401CE
:1032D000460E826F82EC0EF00BEF1DF0078456EC69
:1032E00034F0D5EC2DF02DC500F178EC2DF0040173
:1032F0004C0E826F82EC0EF00401300E826F82EC75
:103300000EF004012C0E826F82EC0EF031C182F4BB
:103310000401300E822782EC0EF032C182F40401E7
:10332000300E822782EC0EF033C182F40401300E9D
:10333000822782EC0EF004012C0E826F82EC0EF0DC
:10334000D5EC2DF02EC500F178EC2DF031C182F4D2
:103350000401300E822782EC0EF032C182F40401A7
:10336000300E822782EC0EF033C182F40401300E5D
:10337000822782EC0EF007940BEF1DF004014C0E37
:10338000826F82EC0EF00401650E826F82EC0EF00B
:103390007BEC30F00BEF1DF004014C0E826F82ECE1
:1033A0000EF00401450E826F82EC0EF092EC30F0CC
:1033B0000BEF1DF004014C0E826F82EC0EF0040145
:1033C000620E826F82EC0EF0C0EC30F00BEF1DF05D
:1033D00004014C0E826F82EC0EF00401420E826FEB
:1033E00082EC0EF0A9EC30F00BEF1DF004014C0E56
:1033F000826F82EC0EF00401760E826F82EC0EF08A
:1034000004012C0E826F82EC0EF010A807D004018C
:10341000310E826F82EC0EF00BEF1DF00401300EC6
:10342000826F82EC0EF00BEF1DF004014C0E826FE8
:1034300082EC0EF004015A0E826F82EC0EF0040151
:103440002C0E826F82EC0EF056EC34F0D5EC2DF0A1
:1034500005012E51130A06E005012E51170A0DE051
:1034600046EF1AF00101000E006F000E016F100E02
:10347000026F000E036F46EF1AF00101000E006F9D
:10348000000E016F000E026F010E036F0101100E9E
:10349000046F000E056F000E066F000E076F0BEC39
:1034A0002DF078EC2DF02AC182F40401300E822731
:1034B00082EC0EF02BC182F40401300E822782ECE4
:1034C0000EF02CC182F40401300E822782EC0EF043
:1034D0002DC182F40401300E822782EC0EF02EC141
:1034E00082F40401300E822782EC0EF02FC182F4A8
:1034F0000401300E822782EC0EF030C182F4040108
:10350000300E822782EC0EF031C182F40401300EBD
:10351000822782EC0EF032C182F40401300E822741
:1035200082EC0EF033C182F40401300E822782EC6B
:103530000EF00BEF1DF0078404014C0E826F82EC3D
:103540000EF00401310E826F82EC0EF004012C0E9D
:10355000826F82EC0EF025C500F126C501F127C56A
:1035600002F128C503F10101100E046F000E056F72
:10357000000E066F000E076F0BEC2DF078EC2DF0AF
:103580002AC182F40401300E822782EC0EF02BC196
:1035900082F40401300E822782EC0EF02CC182F4FA
:1035A0000401300E822782EC0EF02DC182F404015A
:1035B000300E822782EC0EF02EC182F40401300E10
:1035C000822782EC0EF02FC182F40401300E822794
:1035D00082EC0EF030C182F40401300E822782ECBE
:1035E0000EF031C182F40401300E822782EC0EF01D
:1035F00032C182F40401300E822782EC0EF033C116
:1036000082F40401300E822782EC0EF007940BEF57
:103610001DF0078404014C0E826F82EC0EF0040151
:10362000320E826F82EC0EF0AEEC32F007940BEFAC
:103630001DF0078404014C0E826F82EC0EF0040131
:10364000330E826F82EC0EF00BEC33F00794A6EF92
:103650001AF0078404014C0E826F82EC0EF0040114
:10366000340E826F82EC0EF004012C0E826F82EC1D
:103670000EF016EC2EF084C32AF185C32BF186C31D
:103680002CF187C32DF188C32EF189C32FF18AC392
:1036900030F18BC331F18CC332F18DC333F10101B1
:1036A000296B23EC2EF09AEC2DF0100E046F000E17
:1036B000056F000E066F000E076FEBEC2CF000C1DB
:1036C00021F501C122F502C123F503C124F509EC5E
:1036D00034F038C5AFF539C5B0F53AC5B1F53BC5DD
:1036E000B2F53CC5B3F53DC5B4F53EC5B5F50EEC38
:1036F00016F004012C0E826F82EC0EF03FC500F133
:1037000040C501F141C502F142C503F10101000EBE
:10371000046F000E056F010E066F000E076F0BECB5
:103720002DF078EC2DF0296798EF1BF09DEF1BF042
:1037300004012D0E826F82EC0EF030C182F4040180
:10374000300E822782EC0EF031C182F40401300E7B
:10375000822782EC0EF004012E0E826F82EC0EF0B6
:1037600032C182F40401300E822782EC0EF033C1A4
:1037700082F40401300E822782EC0EF004012C0E3C
:10378000826F82EC0EF0D5EC2DF043C500F144C5FC
:1037900001F123EC28F004012C0E826F82EC0EF074
:1037A000D5EC2DF045C500F178EC2DF031C182F457
:1037B0000401300E822782EC0EF032C182F4040143
:1037C000300E822782EC0EF033C182F40401300EF9
:1037D000822782EC0EF004012C0E826F82EC0EF038
:1037E00037C5E8FFE8B806D00401300E826F82ECDE
:1037F0000EF005D00401310E826F82EC0EF00794BA
:103800000BEF1DF016EC2EF085C32AF186C32BF1C9
:1038100087C32CF188C32DF189C32EF18AC32FF100
:103820008BC330F18CC331F18DC332F18EC333F1D0
:103830000101296B23EC2EF09AEC2DF00101010E11
:10384000046F000E056F000E066F000E076FDAECB6
:103850002CF0100E046F000E056F000E066F000EA8
:10386000076FEBEC2CF000C129F501C12AF502C16C
:103870002BF503C12CF535EC32F004014C0E826FB0
:1038800082EC0EF00401460E826F82EC0EF0040111
:103890002C0E826F82EC0EF025C500F126C501F1D9
:1038A00027C502F128C503F10101100E046F000EB7
:1038B000056F000E066F000E076F0BEC2DF078EC15
:1038C0002DF02AC182F40401300E822782EC0EF022
:1038D0002BC182F40401300E822782EC0EF02CC141
:1038E00082F40401300E822782EC0EF02DC182F4A6
:1038F0000401300E822782EC0EF02EC182F4040106
:10390000300E822782EC0EF02FC182F40401300EBB
:10391000822782EC0EF030C182F40401300E82273F
:1039200082EC0EF031C182F40401300E822782EC69
:103930000EF032C182F40401300E822782EC0EF0C8
:1039400033C182F40401300E822782EC0EF00BEFBB
:103950001DF00F980BEC33F03080F9EF26F00401E6
:103960004C0E826F82EC0EF00401350E826F82ECF9
:103970000EF004012C0E826F82EC0EF0D5EC2DF0CF
:103980000784B9C500F1079478EC2DF031C182F4B9
:103990000401300E822782EC0EF032C182F4040161
:1039A000300E822782EC0EF033C182F40401300E17
:1039B000822782EC0EF00BEF1DF0CEEC32F0D5EC4E
:1039C0002DF037C500F178EC2DF004014C0E826F1C
:1039D00082EC0EF00401360E826F82EC0EF00401D0
:1039E0002C0E826F82EC0EF031C182F40401300E95
:1039F000822782EC0EF032C182F40401300E82275D
:103A000082EC0EF033C182F40401300E822782EC86
:103A10000EF00BEF1DF08CEC0EF0F9EF26F0040128
:103A20004C0E826F82EC0EF00401500E826F82EC1D
:103A30000EF004012C0E826F82EC0EF085C32AF189
:103A400086C32BF187C32CF188C32DF189C32EF1D6
:103A50008AC32FF18BC330F18CC331F18DC332F1A6
:103A60008EC333F1010123EC2EF09AEC2DF003010B
:103A70008451530A0DE0030184514D0A38E00401DA
:103A8000780E826F82EC0EF08CEC0EF0F9EF26F0DF
:103A90000401530E826F82EC0EF0250E0C6E00C1F5
:103AA0000BF019EC0BF0260E0C6E01C10BF019ECAB
:103AB0000BF0270E0C6E02C10BF019EC0BF0280E68
:103AC0000C6E03C10BF019EC0BF000C157F501C1EE
:103AD00058F502C159F503C15AF500C15BF501C1A2
:103AE0005CF502C15DF503C15EF5ECEF1DF004016C
:103AF0004D0E826F82EC0EF0290E0C6E00C10BF0A1
:103B000019EC0BF000C15FF500C160F5ECEF1DF0A2
:103B100004014C0E826F82EC0EF00401540E826F91
:103B200082EC0EF004012C0E826F82EC0EF084C346
:103B30002AF185C32BF186C32CF187C32DF188C3ED
:103B40002EF189C32FF18AC330F18BC331F18DC3BC
:103B500032F18EC333F1010123EC2EF09AEC2DF0FB
:103B60000101000E046F000E056F010E066F000EBE
:103B7000076FEBEC2CF0210E0C6E00C10BF019EC72
:103B80000BF0220E0C6E01C10BF019EC0BF0230EA2
:103B90000C6E02C10BF019EC0BF0240E0C6E03C17D
:103BA0000BF019EC0BF000C161F501C162F502C127
:103BB00063F503C164F5ECEF1DF004014C0E826F58
:103BC00082EC0EF00401490E826F82EC0EF00401CB
:103BD0002C0E826F82EC0EF0250E30EC0BF0E8CF4D
:103BE00000F1260E30EC0BF0E8CF01F1270E30EC9F
:103BF0000BF0E8CF02F1280E30EC0BF0E8CF03F128
:103C000078EC2DF03BEC2BF00401730E826F82EC0C
:103C10000EF004012C0E826F82EC0EF0D5EC2DF02C
:103C2000290E30EC0BF0E8CF00F178EC2DF03BECF6
:103C30002BF004016D0E826F82EC0EF004012C0E4D
:103C4000826F82EC0EF05BC500F15CC501F15DC5D1
:103C500002F15EC503F178EC2DF03BEC2BF0040192
:103C6000730E826F82EC0EF004012C0E826F82ECD8
:103C70000EF0D5EC2DF060C500F178EC2DF03BECAA
:103C80002BF004016D0E826F82EC0EF004012C0EFD
:103C9000826F82EC0EF061C500F162C501F163C56F
:103CA00002F164C503F114EC27F004012C0E826FBD
:103CB00082EC0EF08CEC0EF0F9EF26F083C32AF1C3
:103CC00084C32BF185C32CF186C32DF187C32EF15C
:103CD00088C32FF189C330F18AC331F18BC332F12C
:103CE0008CC333F1010123EC2EF09AEC2DF0160E6B
:103CF0000C6E00C10BF019EC0BF0170E0C6E01C12D
:103D00000BF019EC0BF0180E0C6E02C10BF019EC55
:103D10000BF0190E0C6E03C10BF019EC0BF000C187
:103D20008EF101C18FF102C190F103C191F100C187
:103D300092F101C193F102C194F103C195F140EFF9
:103D40001FF083C32AF184C32BF185C32CF186C3F2
:103D50002DF187C32EF188C32FF189C330F18AC3B7
:103D600031F18BC332F18CC333F1010123EC2EF01E
:103D70009AEC2DF000C18EF101C18FF102C190F1DA
:103D800003C191F100C192F101C193F102C194F11B
:103D900003C195F140EF1FF083C32AF184C32BF1D7
:103DA00085C32CF186C32DF187C32EF188C32FF173
:103DB00089C330F18AC331F18CC332F18DC333F141
:103DC000010123EC2EF09AEC2DF00101000E046F9E
:103DD000000E056F010E066F000E076FEBEC2CF066
:103DE0001A0E0C6E00C10BF019EC0BF01B0E0C6ED2
:103DF00001C10BF019EC0BF01C0E0C6E02C10BF0A4
:103E000019EC0BF01D0E0C6E03C10BF019EC0BF04E
:103E100000C196F101C197F102C198F103C199F176
:103E200040EF1FF083C32AF184C32BF185C32CF12B
:103E300086C32DF187C32EF188C32FF189C330F1DA
:103E40008AC331F18CC332F18DC333F1010123EC0C
:103E50002EF09AEC2DF00101000E046F000E056F9C
:103E6000010E066F000E076FEBEC2CF000C196F10F
:103E700001C197F102C198F103C199F140EF1FF020
:103E8000160E30EC0BF0E8CF00F1170E30EC0BF013
:103E9000E8CF01F1180E30EC0BF0E8CF02F1190E6B
:103EA00030EC0BF0E8CF03F178EC2DF03BEC2BF08D
:103EB0000401730E826F82EC0EF004012C0E826FEF
:103EC00082EC0EF08EC100F18FC101F190C102F1C0
:103ED00091C103F178EC2DF03BEC2BF00401730E53
:103EE000826F82EC0EF004012C0E826F82EC0EF0D9
:103EF0001A0E30EC0BF0E8CF00F11B0E30EC0BF09B
:103F0000E8CF01F11C0E30EC0BF0E8CF02F11D0EF2
:103F100030EC0BF0E8CF03F114EC27F004012C0E89
:103F2000826F82EC0EF096C100F197C101F198C149
:103F300002F199C103F114EC27F08CEC0EF0F9EFCB
:103F400026F00401690E826F82EC0EF004012C0E43
:103F5000826F82EC0EF00101040E006F000E016F03
:103F6000000E026F000E036F78EC2DF02CC182F46E
:103F70000401300E822782EC0EF02DC182F4040180
:103F8000300E822782EC0EF02EC182F40401300E36
:103F9000822782EC0EF02FC182F40401300E8227BA
:103FA00082EC0EF030C182F40401300E822782ECE4
:103FB0000EF031C182F40401300E822782EC0EF043
:103FC00032C182F40401300E822782EC0EF033C13C
:103FD00082F40401300E822782EC0EF004012C0ED4
:103FE000826F82EC0EF00101060E006F000E016F71
:103FF000000E026F000E036F78EC2DF02CC182F4DE
:104000000401300E822782EC0EF02DC182F40401EF
:10401000300E822782EC0EF02EC182F40401300EA5
:10402000822782EC0EF02FC182F40401300E822729
:1040300082EC0EF030C182F40401300E822782EC53
:104040000EF031C182F40401300E822782EC0EF0B2
:1040500032C182F40401300E822782EC0EF033C1AB
:1040600082F40401300E822782EC0EF004012C0E43
:10407000826F82EC0EF001013A0E006F000E016FAC
:10408000000E026F000E036F78EC2DF02CC182F44D
:104090000401300E822782EC0EF02DC182F404015F
:1040A000300E822782EC0EF02EC182F40401300E15
:1040B000822782EC0EF02FC182F40401300E822799
:1040C00082EC0EF030C182F40401300E822782ECC3
:1040D0000EF031C182F40401300E822782EC0EF022
:1040E00032C182F40401300E822782EC0EF033C11B
:1040F00082F40401300E822782EC0EF004012C0EB3
:10410000826F82EC0EF0200EF86EF76AF66A0401F8
:104110000900F5CF82F482EC0EF00900F5CF82F4AD
:1041200082EC0EF00900F5CF82F482EC0EF009006B
:10413000F5CF82F482EC0EF00900F5CF82F482EC28
:104140000EF00900F5CF82F482EC0EF00900F5CFF5
:1041500082F482EC0EF00900F5CF82F482EC0EF0CE
:104160008CEC0EF0F9EF26F08351630AD8A4F7EF38
:1041700026F08451610AD8A4F7EF26F085516C0A25
:10418000D8A4F7EF26F08651410A3FE08651440A51
:104190001BE08651420AD8B418EF21F08651350A47
:1041A000D8B483EF28F08651360AD8B4D8EF28F077
:1041B0008651370AD8B441EF29F08651380AD8B46D
:1041C0009FEF29F0F7EF26F00798079A04017A0E7F
:1041D000826F82EC0EF00401780E826F82EC0EF09A
:1041E0000401640E826F82EC0EF00401550E826FA2
:1041F00082EC0EF001EF21F004014C0E826F82EC94
:104200000EF08CEC0EF0F9EF26F00788079A040107
:104210007A0E826F82EC0EF00401410E826F82EC06
:104220000EF00401610E826F82EC0EF0F5EF20F0CB
:104230000798078A04017A0E826F82EC0EF004015F
:10424000420E826F82EC0EF00401610E826F82ECEE
:104250000EF0F5EF20F00101666736EF21F0676799
:1042600036EF21F0686736EF21F0696715D04F67A8
:1042700041EF21F0506741EF21F0516741EF21F00C
:1042800052670AD00101000E006F000E016F000E90
:10429000026F000E036F120011B80AD00101620E06
:1042A000046F010E056F000E066F000E076F09D038
:1042B0000101A70E046F020E056F000E066F000EBF
:1042C000076F66C100F167C101F168C102F169C100
:1042D00003F1DAEC2CF003BFDEEF21F0119A119C10
:1042E0000101000E046FA80E056F550E066F020E39
:1042F000076F66C100F167C101F168C102F169C1D0
:1043000003F166C18AF167C18BF168C18CF169C1A3
:104310008DF1DAEC2CF003BF0BD00101000E8A6F97
:10432000A80E8B6F550E8C6F020E8D6F118A119C2B
:104330000E0E30EC0BF0E8CF18F10F0E30EC0BF056
:10434000E8CF19F1100E30EC0BF0E8CF1AF1110E96
:1043500030EC0BF0E8CF1BF123EC2CF08AC104F118
:104360008BC105F18CC106F18DC107F1DAEC2CF09F
:104370000782E7EC2BF023EC2CF00792E7EC2BF014
:104380008AC100F18BC101F18CC102F18DC103F131
:104390000792E7EC2BF0CC0E046FE00E056F870E52
:1043A000066F050E076FDAEC2CF000C118F101C1A1
:1043B00019F102C11AF103C11BF140D013AAE3EFB6
:1043C00021F0138E139A119C119A0101800E006F37
:1043D0001A0E016F060E026F000E036F4FC104F13B
:1043E00050C105F151C106F152C107F1DAEC2CF0D0
:1043F00003AF05D0D5EC2DF0118C119A12000E0EE2
:1044000030EC0BF0E8CF18F10F0E30EC0BF0E8CFEA
:1044100019F1100E30EC0BF0E8CF1AF1110E30EC60
:104420000BF0E8CF1BF14FC100F150C101F151C1B8
:1044300002F152C103F10782E7EC2BF018C100F141
:1044400019C101F11AC102F11BC103F112000401EB
:10445000730E826F82EC0EF004012C0E826F82ECE0
:104460000EF0078462C166F163C167F164C168F14F
:1044700065C169F14BC14FF14CC150F14DC151F1D2
:104480004EC152F157C159F158C15AF107944DEC40
:1044900022F08CEC0EF0F9EF26F066C100F167C156
:1044A00001F168C102F169C103F1010178EC2DF05D
:1044B0003BEC2BF00401630E826F82EC0EF00401E2
:1044C0002C0E826F82EC0EF04FC100F150C101F151
:1044D00051C102F152C103F1010178EC2DF03BEC26
:1044E0002BF00401660E826F82EC0EF004012C0E9C
:1044F000826F82EC0EF0D5EC2DF059C100F15AC15B
:1045000001F1010178EC2DF03BEC2BF00401740E6D
:10451000826F82EC0EF0120010820401530E826F43
:1045200082EC0EF004012C0E826F82EC0EF083C33D
:104530002AF184C32BF185C32CF186C32DF187C3E7
:104540002EF188C32FF189C330F18AC331F18BC3B7
:1045500032F18CC333F1010123EC2EF09AEC2DF0F3
:1045600000C166F101C167F102C168F103C169F1DF
:104570008EC32AF18FC32BF190C32CF191C32DF17F
:1045800092C32EF193C32FF194C330F195C331F14F
:1045900096C332F197C333F1010123EC2EF09AEC6C
:1045A0002DF000C14FF101C150F102C151F103C121
:1045B00052F116EC2EF099C32FF19AC330F19BC340
:1045C00031F19CC332F19DC333F1010123EC2EF094
:1045D0009AEC2DF000C159F101C15AF14DEC22F0D5
:1045E00004012C0E826F82EC0EF007EF23F0118E87
:1045F00019A002D019AE108C18BE02D018A4108ECB
:1046000003018251520A02E10F8201D00F928251BE
:10461000750A02E1108401D010948251550A02E11A
:10462000108601D010968351310A03E1138213845E
:1046300002D01392139411A003D011A401D01084BE
:10464000078410B285EF23F010A469EF23F0BAC1FC
:1046500066F1BBC167F1BCC168F1BDC169F1BEC102
:104660006AF1BFC16BF1C0C16CF1C1C16DF1C2C1D2
:104670006EF1C3C16FF1C4C170F1C5C171F1C6C1A2
:1046800072F1C7C173F1C8C174F1C9C175F1CAC172
:1046900076F1CBC177F1CCC178F1CDC179F1CEC142
:1046A0007AF1CFC17BF1D0C17CF1D1C17DF1D2C112
:1046B0007EF1D3C17FF1D4C180F1D5C181F1D6C1E2
:1046C00082F1D7C183F1D8C184F1D9C185F171EFED
:1046D00023F062C166F163C167F164C168F165C12D
:1046E00069F1BAC186F1BBC187F1BCC188F1BDC116
:1046F00089F14BC14FF14CC150F14DC151F14EC147
:1047000052F157C159F158C15AF107940FA0A7EFC0
:1047100023F00101966794EF23F0976794EF23F05D
:10472000986794EF23F0996798EF23F0A7EF23F0B1
:104730002BEC21F096C104F197C105F198C106F167
:1047400099C107F1DAEC2CF003BFBDEF26F02BEC9A
:1047500021F00101000E046F000E056F010E066FBF
:10476000000E076F0BEC2DF011A02AD011A228D05B
:1047700078EC2DF0296701D005D004012D0E826F51
:1047800082EC0EF030C182F40401300E822782ECFC
:104790000EF031C182F40401300E822782EC0EF05B
:1047A00032C182F40401300E822782EC0EF033C154
:1047B00082F40401300E822782EC0EF08CEC0EF0B5
:1047C00012A8C5D012981AC01BF01B3A1B42070E44
:1047D0001B1600011B50000AD8B473EF24F000012F
:1047E0001B50010AD8B4FFEF23F000011B50020A4E
:1047F000D8B4FDEF23F0A5EF24F0A5EF24F0D5EC1D
:104800002DF02AC001F12BC000F1D8900133003304
:10481000D890013300330101630E046F000E056F61
:10482000000E066F000E076F0BEC2DF0280E046FC4
:10483000000E056F000E066F000E076FDAEC2CF00D
:1048400000C12DF0D5EC2DF028C001F1019F019D94
:1048500029C000F10101A40E046F000E056F000EC7
:10486000066F000E076F0BEC2DF000C12CF000C19D
:1048700004F101C105F102C106F103C107F1640EA3
:10488000006F000E016F000E026F000E036FDAEC76
:104890002CF0050E046F000E056F000E066F000E63
:1048A000076F0BEC2DF000C104F101C105F102C14D
:1048B00006F103C107F1D5EC2DF02DC000F1DAECC3
:1048C0002CF000C12EF02EC0E8FF050F2D5C03E791
:1048D0008A84A5EF24F02EC0E8FF0A0F2D5C01E6C4
:1048E0008A94A5EF24F000C124F101C125F102C191
:1048F00026F103C127F1D5EC2DF0DBEC2DF01A5099
:104900001F0BE8CF00F10101640E046F000E056F6C
:10491000000E066F000E076FEBEC2CF024C104F1C3
:1049200025C105F126C106F127C107F1DAEC2CF00B
:1049300003BF02D08A9401D08A8424C100F125C12A
:1049400001F126C102F127C103F1F9EF26F000C100
:1049500024F101C125F102C126F103C127F110AEF6
:104960004DD0109E00C108F101C109F102C10AF148
:1049700003C10BF178EC2DF030C1DAF131C1DBF17C
:1049800032C1DCF133C1DDF108C100F109C101F12F
:104990000AC102F10BC103F101016C0E046F070E95
:1049A000056F000E066F000E076FDAEC2CF003BFE8
:1049B00004D00101550EDE6F1CD008C100F109C101
:1049C00001F10AC102F10BC103F10101A40E046F50
:1049D000060E056F000E066F000E076FDAEC2CF066
:1049E00003BF04D001017F0EDE6F03D00101FF0E73
:1049F000DE6F1C8E11AEBDEF26F0119E24C100F1BA
:104A000025C101F126C102F127C103F111A005D092
:104A100011A203D00FB0BDEF26F010A417EF25F0C0
:104A20000401750E826F82EC0EF01CEF25F004017C
:104A3000720E826F82EC0EF004012C0E826F82ECFB
:104A40000EF078EC2DF029672BEF25F00401200EF5
:104A5000826F2EEF25F004012D0E826F82EC0EF096
:104A600030C182F40401300E822782EC0EF031C195
:104A700082F40401300E822782EC0EF004012E0E27
:104A8000826F82EC0EF032C182F40401300E822774
:104A900082EC0EF033C182F40401300E822782ECE6
:104AA0000EF004016D0E826F82EC0EF004012C0EEC
:104AB000826F82EC0EF04FC100F150C101F151C183
:104AC00002F152C103F1010178EC2DF03BEC2BF027
:104AD0000401480E826F82EC0EF004017A0E826FA0
:104AE00082EC0EF004012C0E826F82EC0EF066C197
:104AF00000F167C101F168C102F169C103F101016F
:104B000078EC2DF03BEC2BF00401630E826F82EC0D
:104B10000EF004012C0E826F82EC0EF066C100F1E3
:104B200067C101F168C102F169C103F101010A0E17
:104B3000046F000E056F000E066F000E076FEBECA2
:104B40002CF0000E046F120E056F000E066F000EA3
:104B5000076F0BEC2DF078EC2DF02AC182F40401E4
:104B6000300E822782EC0EF02BC182F40401300E4D
:104B7000822782EC0EF02CC182F40401300E8227D1
:104B800082EC0EF02DC182F40401300E822782ECFB
:104B90000EF02EC182F40401300E822782EC0EF05A
:104BA0002FC182F40401300E822782EC0EF030C156
:104BB00082F40401300E822782EC0EF004012E0EE6
:104BC000826F82EC0EF031C182F40401300E822734
:104BD00082EC0EF032C182F40401300E822782ECA6
:104BE0000EF033C182F40401300E822782EC0EF005
:104BF0000401730E826F82EC0EF004012C0E826FA2
:104C000082EC0EF0D5EC2DF059C100F15AC101F142
:104C100023EC28F013A25CEF26F004012C0E826F27
:104C200082EC0EF086C166F187C167F188C168F138
:104C300089C169F12BEC21F00101000E046F000E17
:104C4000056F010E066F000E076F0BEC2DF078EC70
:104C50002DF0296731EF26F00401200E826F34EF2A
:104C600026F004012D0E826F82EC0EF030C182F42A
:104C70000401300E822782EC0EF031C182F404016F
:104C8000300E822782EC0EF004012E0E826F82EC31
:104C90000EF032C182F40401300E822782EC0EF055
:104CA00033C182F40401300E822782EC0EF004013D
:104CB0006D0E826F82EC0EF013A483EF26F00401D8
:104CC0002C0E826F82EC0EF013AC71EF26F0040113
:104CD000500E826F82EC0EF0139C1398139A83EFA0
:104CE00026F013AE7EEF26F00401460E826F82ECB2
:104CF0000EF0139E1398139A83EF26F00401530EBF
:104D0000826F82EC0EF00FB289EF26F00FA0BBEF9E
:104D100026F004012C0E826F82EC0EF0200EF86E4D
:104D2000F76AF66A04010900F5CF82F482EC0EF00E
:104D30000900F5CF82F482EC0EF00900F5CF82F481
:104D400082EC0EF00900F5CF82F482EC0EF009003F
:104D5000F5CF82F482EC0EF00900F5CF82F482ECFC
:104D60000EF00900F5CF82F482EC0EF00900F5CFC9
:104D700082F482EC0EF08CEC0EF00F90109E1298E4
:104D8000F9EF26F00401630E826F82EC0EF004014D
:104D90002C0E826F82EC0EF0FFEC26F004012C0E3C
:104DA000826F82EC0EF072EC27F004012C0E826F01
:104DB00082EC0EF0EEEC27F004012C0E826F82ECF8
:104DC0000EF00101F80E006FCD0E016F660E026F3E
:104DD000030E036F14EC27F004012C0E826F82EC9B
:104DE0000EF004EC28F08CEC0EF0F9EF26F08CECD1
:104DF0000EF00301C26B0790109208EF2AF0D890D2
:104E00000E0E30EC0BF0E8CF00F10F0E30EC0BF093
:104E1000E8CF01F1100E30EC0BF0E8CF02F1110EEB
:104E200030EC0BF0E8CF03F10101000E046F000E2F
:104E3000056F010E066F000E076F0BEC2DF078EC7E
:104E40002DF02AC182F40401300E822782EC0EF08C
:104E50002BC182F40401300E822782EC0EF02CC1AB
:104E600082F40401300E822782EC0EF02DC182F410
:104E70000401300E822782EC0EF02EC182F4040170
:104E8000300E822782EC0EF02FC182F40401300E26
:104E9000822782EC0EF030C182F40401300E8227AA
:104EA00082EC0EF031C182F40401300E822782ECD4
:104EB0000EF004012E0E826F82EC0EF032C182F4ED
:104EC0000401300E822782EC0EF033C182F404011B
:104ED000300E822782EC0EF004016D0E826F82ECA0
:104EE0000EF01200120E30EC0BF0E8CF00F1130EB2
:104EF00030EC0BF0E8CF01F1140E30EC0BF0E8CF02
:104F000002F1150E30EC0BF0E8CF03F101010A0EAF
:104F1000046F000E056F000E066F000E076FEBECBE
:104F20002CF0000E046F120E056F000E066F000EBF
:104F3000076F0BEC2DF078EC2DF02AC182F4040100
:104F4000300E822782EC0EF02BC182F40401300E69
:104F5000822782EC0EF02CC182F40401300E8227ED
:104F600082EC0EF02DC182F40401300E822782EC17
:104F70000EF02EC182F40401300E822782EC0EF076
:104F80002FC182F40401300E822782EC0EF030C172
:104F900082F40401300E822782EC0EF004012E0E02
:104FA000826F82EC0EF031C182F40401300E822750
:104FB00082EC0EF032C182F40401300E822782ECC2
:104FC0000EF033C182F40401300E822782EC0EF021
:104FD0000401730E826F82EC0EF012000A0E30ECA8
:104FE0000BF0E8CF00F10B0E30EC0BF0E8CF01F145
:104FF0000C0E30EC0BF0E8CF02F10D0E30EC0BF0A4
:10500000E8CF03F123EF28F0060E30EC0BF0E8CFE9
:1050100000F1070E30EC0BF0E8CF01F1080E30EC98
:105020000BF0E8CF02F1090E30EC0BF0E8CF03F102
:1050300023EF28F00101D5EC2DF0078457C100F1D2
:1050400058C101F107940101E80E046F800E056F4D
:10505000000E066F000E076FEBEC2CF0000E046FD5
:10506000040E056F000E066F000E076F0BEC2DF09F
:10507000880E046F130E056F000E066F000E076F8B
:10508000DAEC2CF00A0E046F000E056F000E066FAE
:10509000000E076F0BEC2DF078EC2DF00101296765
:1050A00057EF28F00401200E826F5AEF28F0040118
:1050B0002D0E826F82EC0EF030C182F40401300EAE
:1050C000822782EC0EF031C182F40401300E822777
:1050D00082EC0EF032C182F40401300E822782ECA1
:1050E0000EF004012E0E826F82EC0EF033C182F4BA
:1050F0000401300E822782EC0EF00401430E826F11
:1051000082EC0EF0120087C32AF188C32BF189C309
:105110002CF18AC32DF18BC32EF18CC32FF18DC3DB
:1051200030F18EC331F190C332F191C333F10101FB
:10513000296B23EC2EF09AEC2DF00101000E046F88
:10514000000E056F010E066F000E076FEBEC2CF0E2
:105150000E0E0C6E00C10BF019EC0BF00F0E0C6E66
:1051600001C10BF019EC0BF0100E0C6E02C10BF02C
:1051700019EC0BF0110E0C6E03C10BF019EC0BF0D7
:1051800004017A0E826F82EC0EF004012C0E826F05
:1051900082EC0EF00401350E826F82EC0EF00401F9
:1051A0002C0E826F82EC0EF0FFEC26F001EF21F066
:1051B00087C32AF188C32BF189C32CF18AC32DF14F
:1051C0008BC32EF18CC32FF18DC330F18EC331F11F
:1051D00090C332F191C333F10101296B23EC2EF01E
:1051E0009AEC2DF0880E046F130E056F000E066FFB
:1051F000000E076FDFEC2CF0000E046F040E056F3D
:10520000000E066F000E076FEBEC2CF00101E80EAC
:10521000046F800E056F000E066F000E076F0BEC1B
:105220002DF00A0E0C6E00C10BF019EC0BF00B0EFA
:105230000C6E01C10BF019EC0BF00C0E0C6E02C1E0
:105240000BF019EC0BF00D0E0C6E03C10BF019EC0A
:105250000BF004017A0E826F82EC0EF004012C0E2A
:10526000826F82EC0EF00401360E826F82EC0EF03B
:1052700004012C0E826F82EC0EF0EEEC27F001EFB1
:1052800021F087C32AF188C32BF189C32CF18AC38B
:105290002DF18BC32EF18CC32FF18DC330F18FC351
:1052A00031F190C332F191C333F1010123EC2EF0BF
:1052B0009AEC2DF0000E046F120E056F000E066FB3
:1052C000000E076FEBEC2CF001010A0E046F000ECC
:1052D000056F000E066F000E076F0BEC2DF0120E1F
:1052E0000C6E00C10BF019EC0BF0130E0C6E01C12B
:1052F0000BF019EC0BF0140E0C6E02C10BF019EC54
:105300000BF0150E0C6E03C10BF019EC0BF0040141
:105310007A0E826F82EC0EF004012C0E826F82EC0A
:105320000EF00401370E826F82EC0EF004012C0E99
:10533000826F82EC0EF072EC27F001EF21F087C350
:105340002AF188C32BF189C32CF18AC32DF18BC3B9
:105350002EF18CC32FF18DC330F18EC331F190C388
:1053600032F191C333F10101296B23EC2EF09AEC59
:105370002DF0880E046F130E056F000E066F000EE1
:10538000076FDFEC2CF0000E046F040E056F000EAB
:10539000066F000E076FEBEC2CF00101E80E046FB6
:1053A000800E056F000E066F000E076F0BEC2DF0E0
:1053B000060E0C6E00C10BF019EC0BF0070E0C6E14
:1053C00001C10BF019EC0BF0080E0C6E02C10BF0D2
:1053D00019EC0BF0090E0C6E03C10BF019EC0BF07D
:1053E00004017A0E826F82EC0EF004012C0E826FA3
:1053F00082EC0EF00401380E826F82EC0EF0040194
:105400002C0E826F82EC0EF004EC28F001EF21F0FC
:1054100007A87BEF2AF00101800E006F1A0E016FC2
:10542000060E026F000E036F4BC104F14CC105F173
:105430004DC106F14EC107F1DAEC2CF003BFC1EF0C
:105440002AF035EC2BF04BC100F14CC101F14DC1FC
:1054500002F14EC103F10782E7EC2BF018C104F111
:1054600019C105F11AC106F11BC107F1F80E006F51
:10547000CD0E016F660E026F030E036FDAEC2CF097
:105480000E0E0C6E00C10BF019EC0BF00F0E0C6E33
:1054900001C10BF019EC0BF0100E0C6E02C10BF0F9
:1054A00019EC0BF0110E0C6E03C10BF019EC0BF0A4
:1054B00007840101D5EC2DF057C100F158C101F16D
:1054C00007940A0E0C6E00C10BF019EC0BF00B0EDA
:1054D0000C6E01C10BF019EC0BF00C0E0C6E02C13E
:1054E0000BF019EC0BF00D0E0C6E03C10BF019EC68
:1054F0000BF0C1EF2AF007AAC1EF2AF007840101DF
:10550000D5EC2DF057C100F158C101F10794060EFA
:105510000C6E00C10BF019EC0BF0070E0C6E01C104
:105520000BF019EC0BF0080E0C6E02C10BF019EC2D
:105530000BF0090E0C6E03C10BF019EC0BF0078495
:1055400062C100F163C101F164C102F165C103F1FF
:105550000794120E0C6E00C10BF019EC0BF0130E39
:105560000C6E01C10BF019EC0BF0140E0C6E02C1A5
:105570000BF019EC0BF0150E0C6E03C10BF019ECCF
:105580000BF00798079A0401805181197F0B0DE0F9
:105590009EA8FED714EE00F081517F0BE126E75064
:1055A000812B0F01AD6EC3EF2AF005012F51010AC7
:1055B00013E081AAFDEF2AF005012F51000A0AE04D
:1055C0000FB8ECEF2AF005013067ECEF2AF00FB8C6
:1055D000ECEF2AF095EF34F081B8FDEF2AF005ECFE
:1055E0002FF0FDEF2AF0602FFDEF2AF05FC560F588
:1055F0000501010E306F3C0E316FC9EF0DF018C17F
:1056000000F119C101F11AC102F11BC103F1000E31
:10561000046F000E056F010E066F000E076F0BEC96
:105620002DF029A12AEF2BF02051D8B42AEF2BF02E
:1056300018C100F119C101F11AC102F11BC103F136
:10564000000E046F000E056F0A0E066F000E076F46
:105650000BEC2DF012000101045100130551011350
:10566000065102130751031312000101186B196B45
:105670001A6B1B6B12002AC182F40401300E8227C0
:1056800082EC0EF02BC182F40401300E822782ECF2
:105690000EF02CC182F40401300E822782EC0EF051
:1056A0002DC182F40401300E822782EC0EF02EC14F
:1056B00082F40401300E822782EC0EF02FC182F4B6
:1056C0000401300E822782EC0EF030C182F4040116
:1056D000300E822782EC0EF031C182F40401300ECC
:1056E000822782EC0EF032C182F40401300E822750
:1056F00082EC0EF033C182F40401300E822782EC7A
:105700000EF012002FC182F40401300E822782ECC9
:105710000EF030C182F40401300E822782EC0EF0CC
:1057200031C182F40401300E822782EC0EF032C1C6
:1057300082F40401300E822782EC0EF033C182F431
:105740000401300E822782EC0EF01200060E1E6E4F
:10575000060E1F6E060E206E1E2EACEF2BF01F2EB7
:10576000ACEF2BF0202EACEF2BF08B84020E1E6ED4
:10577000020E1F6E020E206E1E2EBCEF2BF01F2E8F
:10578000BCEF2BF0202EBCEF2BF08B941200FF0E01
:105790001F6E1FC020F0030E1E6E8B841E2ECDEFD9
:1057A0002BF0030E1E6E202ECDEF2BF08B941FC01E
:1057B00020F0030E1E6E1E2EDBEF2BF0030E1E6E6E
:1057C000203EDBEF2BF01F2EC9EF2BF01200010162
:1057D000005305E1015303E1025301E1002BAAEC60
:1057E0002CF0D5EC2DF03951006F3A51016F420E7B
:1057F000046F4B0E056F000E066F000E076FEBEC8B
:105800002CF000C104F101C105F102C106F103C190
:1058100007F118C100F119C101F11AC102F11BC150
:1058200003F107B218EF2CF0DFEC2CF01AEF2CF09C
:10583000DAEC2CF000C118F101C119F102C11AF122
:1058400003C11BF11200D5EC2DF059C100F15AC172
:1058500001F1060E30EC0BF0E8CF04F1070E30EC4E
:105860000BF0E8CF05F1080E30EC0BF0E8CF06F1B5
:10587000090E30EC0BF0E8CF07F1DAEC2CF000C1A8
:1058800024F101C125F102C126F103C127F1290E3E
:10589000046F000E056F000E066F000E076FEBEC35
:1058A0002CF0EE0E046F430E056F000E066F000E17
:1058B000076FDFEC2CF024C104F125C105F126C1EE
:1058C00006F127C107F1EBEC2CF000C11CF101C17E
:1058D0001DF102C11EF103C11FF1120E30EC0BF0DD
:1058E000E8CF04F1130E30EC0BF0E8CF05F1140E05
:1058F00030EC0BF0E8CF06F1150E30EC0BF0E8CFF2
:1059000007F10D0E006F000E016F000E026F000E0A
:10591000036FEBEC2CF0180E046F000E056F000EF9
:10592000066F000E076F0BEC2DF01CC104F11DC1BA
:1059300005F11EC106F11FC107F1DFEC2CF06A0E64
:10594000046F2A0E056F000E066F000E076FDAEC6B
:105950002CF01200BF0EFA6E200E3A6F396BD89001
:105960000037013702370337D8B0BBEF2CF03A2F9E
:10597000B0EF2CF039073A070353D8B412000331C3
:10598000070B80093F6F03390F0B010F396F80EC54
:105990005FF0406F390580EC5FF0405D405F396B30
:1059A0003F33D8B0392739333FA9D0EF2CF04051DD
:1059B000392712000101FAEC2DF0D8B012000101D4
:1059C00003510719346FBDEC2DF0D890075103191E
:1059D00034AF800F12000101346BE1EC2DF0D8A040
:1059E000F7EC2DF0D8B01200CCEC2DF0D5EC2DF06A
:1059F0001F0E366F0DEC2EF00B35D8B0BDEC2DF030
:105A0000D8A00335D8B01200362FFAEF2CF034B1FD
:105A1000E4EC2DF012000101346B04510511061164
:105A200007110008D8A0E1EC2DF0D8A0F7EC2DF07C
:105A3000D8B01200086B096B0A6B0B6B0DEC2EF0E3
:105A40001F0E366F0DEC2EF007510B5DD8A435EF0D
:105A50002DF006510A5DD8A435EF2DF00551095DF2
:105A6000D8A435EF2DF00451085DD8A048EF2DF0F3
:105A70000451085F0551D8A0053D095F0651D8A023
:105A8000063D0A5F0751D8A0073D0B5FD890008103
:105A9000362F22EF2DF034B1E4EC2DF0346BE1EC35
:105AA0002DF0D89011EC2EF007510B5DD8A465EFC6
:105AB0002DF006510A5DD8A465EF2DF00551095D62
:105AC000D8A465EF2DF00451085DD8A074EF2DF037
:105AD000003F74EF2DF0013F74EF2DF0023F74EFA3
:105AE0002DF0032BD8B4120034B1E4EC2DF01200E9
:105AF0000101346BE1EC2DF0D8B0120016EC2EF061
:105B0000200E366F003701370237033711EE33F0BE
:105B10000A0E376FE7360A0EE75CD8B0E76EE5523B
:105B2000372F8AEF2DF0362F82EF2DF034B12981F7
:105B3000D890120001010A0E346F200E366F11EE5C
:105B400029F03451376F0A0ED890E652D8B0E726C4
:105B5000E732372FA5EF2DF0033302330133003343
:105B6000362F9FEF2DF0E750FF0FD8A00335D8B0A8
:105B7000120029B1E4EC2DF0120004510027055168
:105B8000D8B0053D01270651D8B0063D0227075180
:105B9000D8B0073D032712000051086F0151096F6B
:105BA00002510A6F03510B6F12000101006B016B70
:105BB000026B036B12000101046B056B066B076B34
:105BC00012000335D8A012000351800B001F011FE3
:105BD000021F031F003FF4EF2DF0013FF4EF2DF003
:105BE000023FF4EF2DF0032B342B03251200073571
:105BF000D8A012000751800B041F051F061F071FA6
:105C0000043F0AEF2EF0053F0AEF2EF0063F0AEFA1
:105C10002EF0072B342B07251200003701370237EF
:105C20000337083709370A370B3712000101296B90
:105C30002A6B2B6B2C6B2D6B2E6B2F6B306B316BA0
:105C4000326B336B120001012A510F0B2A6F2B515B
:105C50000F0B2B6F2C510F0B2C6F2D510F0B2D6F2A
:105C60002E510F0B2E6F2F510F0B2F6F30510F0B2B
:105C7000306F31510F0B316F32510F0B326F335187
:105C80000F0B336F120010A806D08994000EC76E58
:105C9000220EC66E05D08984000EC76E220EC66E17
:105CA000050EE82EFED7120010A802D0898401D07C
:105CB0008994050EE82EFED7120043EC2EF09E9636
:105CC000C69E000EC96EFF0E9EB602D0E82EFCD70F
:105CD0009E96C69E000EC96EFF0E9EB602D0E82E9E
:105CE000FCD7C9CFAFF59E96C69E000EC96EFF0EBB
:105CF0009EB602D0E82EFCD7C9CFB0F59E96C69EC0
:105D0000000EC96EFF0E9EB602D0E82EFCD7C9CF9A
:105D1000B1F59E96C69E000EC96EFF0E9EB602D0CD
:105D2000E82EFCD7C9CFB2F59E96C69E000EC96E6E
:105D3000FF0E9EB602D0E82EFCD7C9CFB3F59E96D3
:105D4000C69E000EC96EFF0E9EB602D0E82EFCD78E
:105D5000C9CFB4F59E96C69E000EC96EFF0E9EB6C4
:105D600002D0E82EFCD7C9CFB5F554EC2EF01200C6
:105D700043EC2EF09E96C69E800EC96EFF0E9EB618
:105D800002D0E82EFCD79E96C69EAFC5C9FFFF0E77
:105D90009EB602D0E82EFCD79E96C69EB0C5C9FF1F
:105DA000FF0E9EB602D0E82EFCD79E96C69EB1C5C9
:105DB000C9FFFF0E9EB602D0E82EFCD79E96C69E67
:105DC000B2C5C9FFFF0E9EB602D0E82EFCD79E9644
:105DD000C69EB3C5C9FFFF0E9EB602D0E82EFCD703
:105DE0009E96C69EB4C5C9FFFF0E9EB602D0E82E91
:105DF000FCD79E96C69EB5C5C9FFFF0E9EB602D0C3
:105E0000E82EFCD754EC2EF0120043EC2EF09E96B8
:105E1000C69E070EC96EFF0E9EB602D0E82EFCD7B6
:105E20009E96C69E000EC96EFF0E9EB602D0E82E4C
:105E3000FCD7C9CFAFF59E96C69E000EC96EFF0E69
:105E40009EB602D0E82EFCD7C9CFB0F59E96C69E6E
:105E5000000EC96EFF0E9EB602D0E82EFCD7C9CF49
:105E6000B1F59E96C69E000EC96EFF0E9EB602D07C
:105E7000E82EFCD7C9CFB2F554EC2EF043EC2EF04F
:105E80009E96C69E22C0C9FFFF0E9EB602D0E82E87
:105E9000FCD79E96C69E000EC96EFF0E9EB602D01F
:105EA000E82EFCD7C9CFB6F554EC2EF0120043EC27
:105EB0002EF09E96C69E870EC96EFF0E9EB602D02D
:105EC000E82EFCD79E96C69EAFC5C9FFFF0E9EB6B4
:105ED00002D0E82EFCD79E96C69EB0C5C9FFFF0E25
:105EE0009EB602D0E82EFCD79E96C69EB1C5C9FFCD
:105EF000FF0E9EB602D0E82EFCD79E96C69EB2C577
:105F0000C9FFFF0E9EB602D0E82EFCD754EC2EF04F
:105F100043EC2EF09E96C69E23C0C9FFFF0E9EB690
:105F200002D0E82EFCD79E96C69EB6C5C9FFFF0ECE
:105F30009EB602D0E82EFCD754EC2EF0120043ECB3
:105F40002EF09E96C69E870EC96EFF0E9EB602D09C
:105F5000E82EFCD79E96C69E000EC96EFF0E9EB61A
:105F600002D0E82EFCD79E96C69E800EC96EFF0E0C
:105F70009EB602D0E82EFCD79E96C69E800EC96EB5
:105F8000FF0E9EB602D0E82EFCD79E96C69E800ECF
:105F9000C96EFF0E9EB602D0E82EFCD754EC2EF050
:105FA000120043EC2EF09E96C69E870EC96EFF0E21
:105FB0009EB602D0E82EFCD79E96C69E000EC96EF5
:105FC000FF0E9EB602D0E82EFCD79E96C69E000E0F
:105FD000C96EFF0E9EB602D0E82EFCD79E96C69ED6
:105FE000800EC96EFF0E9EB602D0E82EFCD79E969C
:105FF000C69E800EC96EFF0E9EB602D0E82EFCD75C
:1060000054EC2EF0120010A817D043EC2EF09E9600
:10601000C69E8F0EC96EFF0E9EB602D0E82EFCD72C
:106020009E96C69E000EC96EFF0E9EB602D0E82E4A
:10603000FCD754EC2EF0120005EC2FF0120010A843
:106040002DD043EC2EF09E96C69E23C0C9FFFF0EB6
:106050009EB602D0E82EFCD79E96C69E450EC96E0F
:10606000FF0E9EB602D0E82EFCD754EC2EF043EC87
:106070002EF09E96C69E8F0EC96EFF0E9EB602D063
:10608000E82EFCD79E96C69E000EC96EFF0E9EB6E9
:1060900002D0E82EFCD754EC2EF0120043EC2EF088
:1060A0009E96C69E23C0C9FFFF0E9EB602D0E82E64
:1060B000FCD79E96C69E010EC96EFF0E9EB602D0FC
:1060C000E82EFCD754EC2EF043EC2EF09E96C69EA4
:1060D000910EC96EFF0E9EB602D0E82EFCD79E969A
:1060E000C69EA50EC96EFF0E9EB602D0E82EFCD746
:1060F00054EC2EF0120043EC2EF09E96C69E23C068
:10610000C9FFFF0E9EB602D0E82EFCD79E96C69E13
:10611000810EC96EFF0E9EB602D0E82EFCD754EC5D
:106120002EF0120043EC2EF09E96C69E23C0C9FFAF
:10613000FF0E9EB602D0E82EFCD79E96C69E010E9C
:10614000C96EFF0E9EB602D0E82EFCD754EC2EF09E
:10615000120043EC2EF09E96C69E910EC96EFF0E65
:106160009EB602D0E82EFCD79E96C69EA50EC96E9E
:10617000FF0E9EB602D0E82EFCD754EC2EF0120093
:1061800043EC2EF09E96C69E910EC96EFF0E9EB6F3
:1061900002D0E82EFCD79E96C69E000EC96EFF0E5A
:1061A0009EB602D0E82EFCD754EC2EF0120005016A
:1061B000256B266B276B286B899A400EC76E200EC5
:1061C000C66E9E96C69E030EC96EFF0E9EB602D088
:1061D000E82EFCD79E96C69E27C5C9FFFF0E9EB629
:1061E00002D0E82EFCD79E96C69E26C5C9FFFF0E9C
:1061F0009EB602D0E82EFCD79E96C69E25C5C9FF46
:10620000FF0E9EB602D0E82EFCD79E96C69EC952BF
:10621000FF0E9EB602D0E82EFCD7898A0F01C95026
:10622000FF0A01E1120005012E51130A05E00501E4
:106230002E51170A0CE012000501F00E256FFF0E1B
:10624000266F0F0E276F000E286F30EF31F005011B
:10625000F00E256FFF0E266FFF0E276F000E286FC2
:10626000899A400EC76E200EC66E9E96C69E030E7D
:10627000C96EFF0E9EB602D0E82EFCD79E96C69E33
:1062800027C5C9FFFF0E9EB602D0E82EFCD79E960A
:10629000C69E26C5C9FFFF0E9EB602D0E82EFCD7CB
:1062A0009E96C69E25C5C9FFFF0E9EB602D0E82E5B
:1062B000FCD79E96C69EC952FF0E9EB602D0E82E0F
:1062C000FCD7898A0F01C950FF0A1DE005012E5134
:1062D000130A05E005012E51170A0BE01200050113
:1062E000000E256F000E266F100E276F000E286F10
:1062F00012000501000E256F000E266F000E276F9D
:10630000010E286F12000501256B266B276B286B89
:1063100005012E51130A05E005012E51170A0CE064
:1063200012000501000E216F000E226F080E236F70
:10633000000E246FA5EF31F00501000E216F000E55
:10634000226F800E236F000E246F21C500F122C53D
:1063500001F123C502F124C503F125C504F126C5C9
:1063600005F127C506F128C507F12BEC2BF000C17C
:1063700025F501C126F502C127F503C128F5899A43
:10638000400EC76E200EC66E9E96C69E030EC96E48
:10639000FF0E9EB602D0E82EFCD79E96C69E27C55D
:1063A000C9FFFF0E9EB602D0E82EFCD79E96C69E71
:1063B00026C5C9FFFF0E9EB602D0E82EFCD79E96DA
:1063C000C69E25C5C9FFFF0E9EB602D0E82EFCD79B
:1063D0009E96C69EC952FF0E9EB602D0E82EFCD7EE
:1063E000898AC950FF0A08E104C125F505C126F5CF
:1063F00006C127F507C128F5D890050124332333BA
:10640000223321332151F00B216F21670FEF32F03E
:1064100022670FEF32F023670FEF32F02467A5EF0A
:1064200031F00501100E2527E86A2623E86A2723A4
:10643000E86A28231200E86A05012E51130A06E0D3
:1064400005012E51170A0BE0020E1200050128511A
:10645000000A03E12751F00B07E0010E12000501CD
:106460002851000A01E0010E120029C500F12AC5D9
:1064700001F12BC502F12CC503F125C504F126C598
:1064800005F127C506F128C507F1DAEC2CF003BFAA
:1064900012001BEC32F0D8A4ADEF32F0899A400E16
:1064A000C76E200EC66E9E96C69E060EC96EFF0E65
:1064B0009EB602D0E82EFCD7898A899A9E96C69EFF
:1064C000020EC96EFF0E9EB602D0E82EFCD79E9635
:1064D000C69E27C5C9FFFF0E9EB602D0E82EFCD788
:1064E0009E96C69E26C5C9FFFF0E9EB602D0E82E18
:1064F000FCD79E96C69E25C5C9FFFF0E9EB602D04C
:10650000E82EFCD79E96C69E000EC96EFF0E9EB664
:1065100002D0E82EFCD7898A899A9E96C69E050EDF
:10652000C96EFF0E9EB602D0E82EFCD79E96C69E80
:10653000C952FF0E9EB602D0E82EFCD7C9B096EF26
:1065400032F0898A0501100E2527E86A2623E86AB9
:106550002723E86A282335EF32F01200899A400E8B
:10656000C76E200EC66E9E96C69E060EC96EFF0EA4
:106570009EB602D0E82EFCD7898A899A9E96C69E3E
:10658000C70EC96EFF0E9EB602D0E82EFCD7898AD0
:106590000501256B266B276B286B1200899A400E2C
:1065A000C76E200EC66E9E96C69E050EC96EFF0E65
:1065B0009EB602D0E82EFCD79E96C69EC952FF0E0C
:1065C0009EB602D0E82EFCD7C9CF37F5898A1200D3
:1065D000899A400EC76E200EC66E9E96C69EB90E54
:1065E000C96EFF0E9EB602D0E82EFCD7898A120033
:1065F000899A400EC76E200EC66E9E96C69EAB0E42
:10660000C96EFF0E9EB602D0E82EFCD7898AFF0E17
:10661000E82EFED712001BEC32F0D8A41200899AA3
:10662000400EC76E200EC66E9E96C69E030EC96EA5
:10663000FF0E9EB602D0E82EFCD79E96C69E27C5BA
:10664000C9FFFF0E9EB602D0E82EFCD79E96C69ECE
:1066500026C5C9FFFF0E9EB602D0E82EFCD79E9637
:10666000C69E25C5C9FFFF0E9EB602D0E82EFCD7F8
:106670009E96C69EC952FF0E9EB602D0E82EFCD74B
:10668000898A0F01C950FF0AD8A408EF34F0050128
:10669000FE0E376F30A037995DEC2EF0AFC538F5A0
:1066A000B0C539F5B1C53AF5B2C53BF5B3C53CF552
:1066B000B4C53DF5B5C53EF50784BAC166F1BBC1A9
:1066C00067F1BCC168F1BDC169F14BC14FF14CC16B
:1066D00050F14DC151F14EC152F157C159F158C15C
:1066E0005AF12BEC21F000C13FF501C140F502C188
:1066F00041F503C142F50501616786EF33F062673A
:1067000086EF33F0636786EF33F064678AEF33F028
:1067100097EF33F061C504F162C505F163C506F179
:1067200064C507F1DAEC2CF003BF08EF34F059C16F
:1067300043F55AC144F5B9C545F5BAC546F50794C0
:106740000501110E326F899A400EC76E200EC66E7B
:106750009E96C69E060EC96EFF0E9EB602D0E82E0D
:10676000FCD7898A899A9E96C69E020EC96EFF0E34
:106770009EB602D0E82EFCD79E96C69E27C5C9FFBE
:10678000FF0E9EB602D0E82EFCD79E96C69E26C56A
:10679000C9FFFF0E9EB602D0E82EFCD79E96C69E7D
:1067A00025C5C9FFFF0E9EB602D0E82EFCD725EE08
:1067B00037F0322F02D0E8EF33F09E96C69EDECF40
:1067C000C9FFFF0E9EB602D0E82EFCD7D9EF33F0FA
:1067D000898A899A9E96C69E050EC96EFF0E9EB640
:1067E00002D0E82EFCD79E96C69EC952FF0E9EB6DA
:1067F00002D0E82EFCD7C9B0F3EF33F0898A050147
:10680000100E2527E86A2623E86A2723E86A28234A
:10681000120021C500F122C501F123C502F124C5F2
:1068200003F1899A400EC76E200EC66E9E96C69ED4
:106830000B0EC96EFF0E9EB602D0E82EFCD79E96B8
:10684000C69E02C1C9FFFF0E9EB602D0E82EFCD73D
:106850009E96C69E01C1C9FFFF0E9EB602D0E82ECD
:10686000FCD79E96C69E00C1C9FFFF0E9EB602D001
:10687000E82EFCD79E96C69EC952FF0E9EB602D049
:10688000E82EFCD725EE37F00501100E326F9E96EC
:10689000C69EC952FF0E9EB602D0E82EFCD7C9CFC5
:1068A000DEFF322F47EF34F0898A1200899A400EBA
:1068B000C76E200EC66E9E96C69E900EC96EFF0EC7
:1068C0009EB602D0E82EFCD79E96C69E000EC96EDC
:1068D000FF0E9EB602D0E82EFCD79E96C69E000EF6
:1068E000C96EFF0E9EB602D0E82EFCD79E96C69EBD
:1068F000000EC96EFF0E9EB602D0E82EFCD79E9603
:10690000C69EC952FF0E9EB602D0E82EFCD7C9CF54
:106910002DF59E96C69EC952FF0E9EB602D0E82E59
:10692000FCD7C9CF2EF5898A1200A6EC2BF0B9C589
:10693000E8FFD70802E3A6EC2BF0B9C5E8FFC808CA
:1069400002E3A6EC2BF0B9C5E8FFB90802E3A6EC18
:106950002BF0B9C5E8FFAA0802E3A6EC2BF0B9C5F5
:10696000E8FF9B0802E3A6EC2BF0E8EC32F0F29C87
:10697000F29E8B94C69AC2909482948C720ED36EBF
:10698000D3A4FED789968A909390F29AF2949D9020
:106990009E909D929E92F298F29203EC30F0FF0E40
:1069A000E8CF00F0E82EFED7002EFCD7F290F2865A
:1069B000815081A8DEEF34F0F29E0300700ED36E9A
:1069C000F296F290010E306E0380C7EC2BF065EF6B
:0269D0000BF0CA
:10BF0000E844F926000C160C2B0C3F0C520C640C68
:10BF1000760C860C960CA50CB30CC10CCF0CDC0C6B
:06BF2000E80CF40C000C1B
:0200000400F00A
:0100C800FE39
:00000001FF
